:020000041100E9
:103000007FB50023284C294D03932800217C284AB2
:1030100001F0CFFA002812D103232800217C03AA53
:1030200001F06EFA00280AD1224B039A9A4206D187
:10303000214B2248E360224B636104B070BD02263D
:10304000217CFE2228001F4B009601F02BFA00285D
:1030500001D00020F1E71C4BA2899A42F9D1217CD2
:10306000FF222800194B009601F01CFA0028F0D12D
:10307000E389174A934203D1164B17486361DCE793
:10308000164A9342E5D1164B164A1B68934206D95D
:10309000C02304222800217C9B0001F06CFA124B13
:1030A00012486361C9E7C046A061FF1FD441FF1FFA
:1030B00081370000595953005959832058BE0011D7
:1030C000E5410011AC61FF1F59590000AE61FF1FBF
:1030D000830500009941001138BE001182150000DF
:1030E000C461FF1F87130000A142001148BE0011F8
:1030F000002370B51A4E1B4C30006361637401F0FD
:103100007FF9402323744B2B0CD9CC233821AC22DC
:1031100030009B01217401F02EFA00280AD000250E
:1031200025740CE0FFF76CFF051E08D1237C0433E7
:10313000DBB2E7E70C4B0D4D63610D4BE381236878
:10314000002B08D1002D06D00C222900200008F009
:1031500057FC2B7B6374300001F090F970BDC046C2
:10316000D441FF1FA061FF1F3942001128BE00118A
:10317000AAAAFFFFF7B5164B0192C318021D002043
:10318000009388235B05D3181B685C1C1AD09CB283
:10319000402C18D88D781E0CAC466746CD782D0291
:1031A0003D43AE4206D1019800280ED110000C70AC
:1031B000240A4C7003249BB20733A343D218009B0C
:1031C0009A42DED3FEBD4432F9E71000FAE7C0466A
:1031D000FC0F0000802213B503000324019189B283
:1031E000520107319B18A14304305A1A88235B050A
:1031F000C3181B68591C03D190429241104016BD60
:1032000099B2402907D80B000733A343C018904256
:10321000ECD30020F3E74430F9E7134B134A1B6863
:10322000126810B5FA24934201D81A00F824104B02
:10323000E4021B689A4210D813000E4A12689A42A0
:103240000ED3013307D1F823DB029C4203D10A4994
:10325000054808F005FD200010BDFC24E402ECE761
:10326000FE24E402F7E7C04600C0071100D00711B2
:1032700000E0071100F00711FFFFFF7FF0B59BB0E2
:10328000150004900391402A00D9A0E006AB5980B4
:103290001A80FFF7C2FF0400042816D9002206A9ED
:1032A000FFF768FF052810D906AB1B88AB420CD18D
:1032B000002D07D0514B2A000499C01808F088FB54
:1032C000002802D101201BB0F0BD06AB1D802000FC
:1032D0000699FFF77FFF041E7BD1069B0793FFF73C
:1032E0009CFF80235B01C618802307001B039E42BE
:1032F00001D3F826F60288235B05F31801931B68B7
:10330000013302D0019808F06BFA3D49019808F0AA
:10331000A7FC3B1D0293331D05938822029B520597
:103320009B181B6808935A1C3CD044219AB2009108
:10333000402A04D80320D11D814389B2009103990A
:103340001B0C8B4224D0402A22D80122300008A92D
:10335000FFF710FF021E1BD1380008A9FFF70AFF74
:103360000400042831D9009A059B9B188022520141
:10337000B218934240D288235B05C118009A09A86D
:1033800008F03EFB1D4B009A09A9F01808F040FB1D
:10339000009A029B9446634402931A4B029AFB18CC
:1033A0009A42BAD388235B05FC1821680198013939
:1033B00008F056FC200008F013FA039A07AB5A8075
:1033C00030000799FFF706FF0400002C03D100200E
:1033D00079E70428FBD988235B05E018069908F0F3
:1033E0003FFC0323EA1C9A4300D16BE7034B04998B
:1033F000E01808F00DFB65E70424ECE70400001179
:10340000FFFFFF7FF80F0000F7B505001400402A0A
:1034100021D8002701AE71803780FFF7FEFE042817
:1034200016D93A003100FFF7A5FE042810D93688D6
:10343000BC420BD0BD4209D0221CB44200D9321C80
:10344000064B92B2C118280008F0DAFA30B2FEBD7D
:10345000C04300B2FBE703204042F8E7040000113C
:1034600037B5042204000D0001A81649FFF7CCFF70
:10347000020004280BD1019BA34208D3AB4204D025
:10348000104901A80195FFF7F9FE01203EBD0E4C41
:1034900023682000019308F0A3F901992000013965
:1034A000019108F0DDFB80235B01E418074B9C428F
:1034B000EED10422034901A80195FFF7DFFE0020A9
:1034C000E4E7C0465555000000C007110000081190
:1034D00030B589B008F034FB10226946254808F061
:1034E0000FF9254B009A9A420ED1019B029A0F2B9D
:1034F00033D8002101240698013B08D2002900D0CE
:103500000292029B013331D10023029325E0551C26
:10351000F2D102002100EFE710341022200004A9AC
:1035200008F0EEF8029B013301D1069B0293882339
:1035300004995B05C918059B06981A03120B0491A0
:103540000592814203D02B4201D108F059FA019B28
:10355000013B0193019B002BDED1029B002B03D08A
:10356000049304984168084709B030BDE025014C38
:103570002D03EFE700000111504859368022F8B5BD
:10358000964C974BD200002120001C6008F0A0FB55
:103590002300944A88331A60934B1A786A23002ACE
:1035A00000D01133E3620A232365904B37221B7846
:1035B0000820A3638E4B2118E361102323628D4BF7
:1035C0003B256361C823DB00A36123008C331A60B1
:1035D0002823013AE26320646364CA67043A211D28
:1035E000CA672100BC310D602100C0310860210094
:1035F000C4310B6021000635CC310D602100083D3F
:10360000C8310D602100D0310A602200D432106030
:103610002200D832136022000227E0322100176016
:103620004222DC310A6021001B3DE4310D602100A3
:10363000E83108602100EC310B6023000521F433F0
:1036400019602300F0331A602300183290331A6097
:1036500023009433186023001E3A98331A60AF2376
:10366000DB002360644BFA262363644B644DE36004
:10367000644BF031A3642300FF31FC33B600A1603A
:1036800021611E60A5627325E5656D3D6565A565D3
:1036900096255D4AAD00E264666258606766A5667D
:1036A00000270925A767E566584F594D6067200038
:1036B0002567E2673A6015279C30676007001A208B
:1036C00038602000A0300700212038602000A8309A
:1036D00007004C4838602000F83006602600642758
:1036E000A436376026005F3FAC3637602600033FC4
:1036F000B03637602600C637B4363760260000275C
:10370000B836376038269E60424E96205E64424E40
:103710005A66DE61414E9A645E62F53EFF3E9E62ED
:103720001E269A67354A8000DE661F675F67DD6583
:103730001D661862DA67BE23394A5B00E250394BD6
:10374000D838235004302250C4225200A350C6233C
:10375000E4205B00E1500433334AE1503349344BF9
:10376000D1603449800019503349E938FF38195085
:1037700032490430195032493248D161324911631B
:10378000324951631900F4310860CE2030494000BD
:1037900011603049195019002F48F83108602F493D
:1037A000D16582212E4A89005A501A002D490832CB
:1037B000D1671A002C49B432116088212B4A890044
:1037C0005A501A002A49883211602A4ADA6408F0ED
:1037D0009FF9012008F034F9F8BDC0460004FF1F2E
:1037E0004464FF1F106FFF1F1044FF1F4A0AFF1F92
:1037F0003A07000080C3C9019A020000DC050000FE
:103800006A18000050C3000088130000F009FF1F71
:10381000204E00006509FF1F68100000C409000069
:1038200040420F0010270000FC00FF1F791CFF1F03
:103830000000FF1FCD2CFF1F5530FF1FED2EFF1F77
:103840003920FF1F2927FF1F5520FF1F0122FF1FBF
:10385000C51FFF1F4D29FF1F352AFF1F9119FF1F8D
:103860005928FF1F7D25FF1F8925FF1FC51EFF1F2C
:103870007D1FFF1F3D1EFF1F0223F0B50124604D79
:10388000604E2B70604B91B01C70604F0393336897
:1038900000212000FB7006F041FE200006F038FDFC
:1038A0000023984205D0FA78552A02D0332A00D056
:1038B00099E03360042006F099FF08F059F9FFF70A
:1038C0005DFE08F045F91F2201240021504B10AE87
:1038D0001A70504B1C70504B1970504B1968914323
:1038E000163A0A431A60602219689143403A0A4323
:1038F0001A6007F0ADFF07F0FBFF494B9847C12066
:10390000FF21484B80001A588A431A50C522920062
:1039100098588843BF390143995098584249084004
:103920008021C9010143802099509958C00509029E
:10393000090A0143995080213C48490107F008FFDA
:10394000032322003A49019400933A4808F0B0F961
:103950002C22394905A808F053F805AC6178207885
:10396000023406F0F5FCA642F8D1344C344B226800
:1039700003201A40A023DB02134323608023226824
:103980009B041343236022682E4B1A4080239B0321
:10399000134323602C4A2D4B934200D8012007F09B
:1039A000DFFE07F0CDFE80232268DB041343236093
:1039B000287808F08DF8039B1878C0B207F0C8FF8C
:1039C00007F0DEFE2249042007F0AAFE06F0DAFE28
:1039D00000F040F800F022FE00F0CAFE00F00AFA03
:1039E000002011B0F0BD00932100194A042007F017
:1039F000DFFE8023DB059C62FFF76AFD5AE7C046C5
:103A00004A0AFF1F34F000401044FF1FD061FF1F1F
:103A1000480AFF1F490AFF1F680AFF1FBCF0004049
:103A2000E1A2000000E100E0FF00FFFF1444FF1FDF
:103A30009856FF1F1454FF1F50BD001114F0004092
:103A4000FF7FF8FFFFFF9FFF0080FF1F106FFF1F2A
:103A50003B000108002210B51100112007F0C8FE3C
:103A600010BD0000F8B500230926364F364C3B62E6
:103A7000E3681120B343E36007F00AFF112007F069
:103A80007FFF112008F0E4F840232268102513433B
:103A9000236080236268DB02134363608023A26893
:103AA00002211343A360A368284A08201340A3609F
:103AB0008023A2689B0113430122A360236CAB43C4
:103AC0002364236C1343236480231B013B62226B1A
:103AD0001F4B1A402263626B1A406263A26B1A404A
:103AE000A263E26B1340E363E3681A4A1340E360A6
:103AF00006F02EFC0121082006F03EFD8023164A28
:103B00005B00516C11200B43536407F0C1FFFD2192
:103B1000C720124B124A89005A50A36B80002B43D6
:103B2000A363E3680F4A3343E3600F4B1958114016
:103B3000802212020A431A50802292051A600B4B0F
:103B40005D63F8BD00F000403CF00040FFFFDFFF88
:103B5000EFFFEFFFFFFF7FFF003800400000FF1F77
:103B60005118FF1FFF00FFFF00E100E000000540CB
:103B700070B5284C238C002B23D0228A002A21D117
:103B8000DA0023826382A382E38223836383A38395
:103B9000E38322606260A260E2601F4D1F4A6420DE
:103BA000EB8093420AD8FA220020D200934205D932
:103BB0001B4A0A21981808F01BF8C0B2002328728B
:103BC000238470BD0720E11CCA7F01320240CA77FE
:103BD00005D10325201DC17F01312940C17708325D
:103BE0005200A352002321001A00088A01321B1838
:103BF0000231082AF9D1221DD27F9200A3506268B7
:103C000023689B18A2689B18E2689B185B099BB20B
:103C1000C3E7C0461061FF1FB861FF1FB70B00006C
:103C200030F8FFFF30B503A804880B20002C0ED11C
:103C30004968074D08784978090201430A20A942DA
:103C400005D1012120001980024B1B7A137030BD71
:103C5000192A0000B861FF1FF7B5150008AA1688D9
:103C60004A680F4F14785278120222430A24BA424B
:103C700014D10122DBB2019200962A0007F0D2FC97
:103C8000041E0BD1074B1B68002B07D068782A78DD
:103C90000002104342425041013098472000FEBDCF
:103CA000022900003C61FF1F30B5012503790400A3
:103CB000BFB02B4211D00A49408807F01FF82842B4
:103CC0000BD0084B01A95B8D4D800B80064B002269
:103CD0001B7A60880B7104F003F93FB030BDC04619
:103CE0003461FF1F4840FF1FB861FF1F10B5054931
:103CF000054806F0B9FF0421044A054806F076FF9E
:103D000010BDC0463461FF1FFFFF00007CBD0011E5
:103D10004840FF1F10B5024804F064FF10BDC046C4
:103D2000A93C0011012303700B4B1A7A4270022246
:103D300082709A78C270DA780271032242711A791D
:103D400082715A79C2710C2202729A794272DB79BD
:103D500083720B207047C046B861FF1F022310B565
:103D60000370013B43700533837010330371443B90
:103D700043712A3383714433C37100230372064BAA
:103D800004001B8843720A30FFF7CCFF831D0A3002
:103D9000C0B2E37010BDC046B861FF1F10B514205B
:103DA00007F0FEFC124B14220021186007F090FF70
:103DB000002007F055FE012007F002FE022007F068
:103DC0006FFD032004F0B2F9042006F0C7F90520C6
:103DD00003F0F0FB062004F0BDF8072001F0A0FA84
:103DE000082006F0E3FE092001F07AF810BDC04675
:103DF0004061FF1F07F09CFE012007F029FE07F03D
:103E0000C7FE0000094B10B50400984205D00129F7
:103E100004D12000064906F027FF10BD0229FCD17D
:103E2000013904F09DFE0028F3D0F6E7FEFF000004
:103E30006661FF1F70B50D7A100004AA2C00168869
:103E400010221440154220D1002E20D10A78022AD7
:103E500018D14A68517815780E4A090229439142CF
:103E600005D00D4A914209D01C800A2404E0142296
:103E70000A491A8007F0C4FD200070BD0C220849D1
:103E80001A80F7E71C800124F6E70824F4E70B24E6
:103E9000F2E7C046F3FF0000F4FF00009C42FF1F62
:103EA00074BE001110B504000749084806F0DCFE96
:103EB000074804F0D7FD0020E40704D50721054A90
:103EC000054806F093FE10BD6661FF1FFFFF00006E
:103ED000053E0011C0BD00118C40FF1F00B50C4B0A
:103EE000BFB01A780B4902A800F0FCFC6B4680B208
:103EF000D880002809D06A46074B01A91B88938007
:103F0000064B0022188803F0EBFF3FB000BDC0460F
:103F10004461FF1F4561FF1FE640FF1FF041FF1F87
:103F200000B50C4BBFB01A780B4902A801F01EFF78
:103F30006B4680B2D880002809D06A46074B01A999
:103F40005B8D9380064B0022188803F0C9FF3FB0B9
:103F500000BDC0466E61FF1F6F61FF1F8C40FF1FD9
:103F6000F041FF1FF7B50E00377A1C0008AB1100B7
:103F70003D001A8820231D401F423CD13378022B7C
:103F80003BD173681F785B781B023B431E4FBB42DB
:103F900008D01E4FBB4214D01D4DAB4221D00A2584
:103FA0002800FEBD002A2AD1142C2AD82200F0684D
:103FB00007F026FD174B1C70012CF1D9FFF7B0FF5D
:103FC000EEE7002A1BD1202C1BD82200F06807F056
:103FD00017FD114B04211C70104B187807F008FDD9
:103FE000DEE7E3B20124009201940A00310007F0F9
:103FF00019FB0500D4E70825D2E70125D0E70B25FA
:10400000CEE70D25CCE7C046F3FF0000F4FF00002B
:10401000022900006E61FF1F4461FF1FF061FF1F56
:10402000332310B5040003700A220749013007F05A
:10403000E7FC064B0F201B681A0AE37222731A0C66
:104040001B0E6273A37310BDB861FF1FE061FF1FF9
:1040500030B5012503790400BFB02B4213D00B49C2
:10406000408806F04BFE28420DD06A46084B02A855
:104070001B889380FFF7D4FF6B46D88000226088AE
:1040800001A903F02DFF3FB030BDC0466661FF1FA0
:10409000E640FF1F10B5024804F0A4FD10BDC04665
:1040A0005140001170B5160004AA148805AA1578AD
:1040B0004A685078117800022A4A08438018052877
:1040C0004BD807F07DFB03131E29343F0720032C38
:1040D0000BD80422121BAA4200D92A0022491A80B6
:1040E0003000091907F08CFC002070BD0720112C4E
:1040F000FBD81222121BAA4200D92A001B491A809F
:10410000EEE707200E2CF0D80F22121BAA4200D98E
:104110002A0017491A80E3E70720032CE5D8042278
:10412000121BAA4200D92A0012491A80D8E7072098
:10413000032CDAD80422121BAA4200D92A000E4905
:104140001A80CDE70720032CCFD80422121BAA42E5
:1041500000D92A0009491A80C2E700220A201A80E1
:10416000C3E7C046DCD5FFFF0BBE00118C61FF1F0B
:10417000FBBD0011F6BD0011F1BD0011ECBD001139
:1041800010B50D21024A034806F030FD10BDC046AF
:10419000E0BD0011FC40FF1F13B5104C0423217C2F
:1041A00001AA00F0ADF9002815D16B469A88236862
:1041B00052BA92B25343228909491B0C9B184B8077
:1041C0006B46DA88636852BA92B2534362891B0C19
:1041D0009B188B8016BD0120FCE7C046A061FF1F25
:1041E000B861FF1F13B5124C06236A46217C00F00C
:1041F00087F9002819D16B461988236849BA89B212
:104200004B4321890B4A1B0C5B1853806B46D978B2
:1042100003335B781B020B435BBA61689BB24B4371
:1042200061891B0C5B18938016BD0120FCE7C0461A
:10423000A061FF1FB861FF1F37B5174C07236A46FF
:10424000217C00F05DF9002824D16B461B787F2B80
:1042500020D86B46DD78F0232A041B031A406B46F6
:104260009B880E495BBA9BB21A4323682D095343BE
:1042700022891B0C9B184B806B465A789B78120343
:104280001B011A4363682A43534362891B0C9B1822
:104290008B803EBD0120FCE7A061FF1FB861FF1FBE
:1042A0007FB50226154C0022217C03AB0096050049
:1042B00000F0F8F8002802D0012004B070BD0E23F1
:1042C000217C0122280000966B4400F0EBF80028C6
:1042D000F2D16B469A892368D2BA5343228908499E
:1042E0001B149B184B806B46DA89636852BA92B2F2
:1042F000534362891B0C9B188B80DEE7A061FF1F74
:10430000B861FF1F70B5184C237C002B0FD0382BE1
:104310000ED1164D280000F073F8CC23AC222800F3
:10432000217C9B0100F027F9280000F0A7F870BD60
:10433000E3890F4A934209D10C4D280000F060F840
:1043400000222800217C00F005F9EDE7094A93429C
:10435000EDD1064D280000F053F890222800217C72
:10436000920100F026F9DFE7A061FF1FD441FF1F93
:10437000830500008320000070B5144C237C002BC3
:104380001FD06369002B1CD0114D280000F038F8B5
:104390006369280098470400280000F06FF8002C9B
:1043A00010D10C4B0422995E002905DA9C801A88F2
:1043B00001321A80200070BD074A9142F7DD9A80D1
:1043C000F5E70124FEF794FEF4E7C046A061FF1F65
:1043D000D441FF1FB861FF1F0F27000010B58024D4
:1043E000064AA4001168436B234205D113685B1A87
:1043F000032BF8D9012010BD0020FCE76008FF1F47
:1044000070B5C17905000C00631E9C411A4BE40293
:10441000E41849000460C9B2007906F0E3F8E979CC
:10442000687949000131C9B206F0DCF8E879093051
:10443000C0B207F00DFC0023E36661332360AA7964
:104440005B3B002A0ED022689A43023B1343236051
:104450000A23E3610733236200232363A363013349
:10446000E36370BD22689A4302231343236046230B
:1044700063610633A361EFE70050004070B500258B
:1044800004000368DD66C0790930C0B207F000FAA5
:104490002900207906F042F82900607906F03EF8FC
:1044A00070BD0000F8B51E0006AB1D78002304683F
:1044B0001700E366616007F043FB01238022E36697
:1044C0002B0027615200013B08D207F0E9FB0820CE
:1044D0000A4A1168002D03D12800F8BD2261F2E7D5
:1044E000236F034203D02369013D33700136136803
:1044F0005B1A032BEED90125EEE7C0466008FF1FCB
:1045000070B51C00002305681600EB66696007F0B3
:1045100017FB01238022EB6623005200013B08D2E7
:1045200007F0BEFB08200A4A1168002C03D12000C6
:1045300070BD2A61F2E72B6F034203D02B69013C67
:104540003370013613685B1A032BEED90124EEE7B2
:104550006008FF1F002370B504681500E366616002
:1045600007F0EEFA0123E366256107F099FB2000CE
:10457000FFF734FF70BD70B51D00002304681600FE
:10458000E366616007F0DCFA0123E36626610F331E
:10459000626B1A42FCD02B0A23611023626B1A4211
:1045A000FCD0EDB2256107F07BFB2000FFF716FF82
:1045B00070BD002370B504681500E366616007F004
:1045C000BFFA0123E3662B0A23611023626B1A42B0
:1045D000FCD0EDB2256107F063FB2000FFF7FEFE83
:1045E00070BD70B51E00002305681400EB6669609D
:1045F00007F0A6FA0123A619EB660F33B44205D1E2
:1046000007F04EFB2800FFF7E9FE70BD2178296115
:10461000696B1942FCD00134F0E7000010B5084C7A
:10462000E368002B08D18022064B52021B689B18BE
:104630006360054B1B68236007F01AF9A06010BD8A
:10464000E061FF1FC8F00040CCF0004070B5184A90
:10465000936A916A9942FBD116498A689A421FD39C
:104660009A1A8B60144B0126186893B2D202D20EAC
:104670004343424300204C681B0A1B1912029B183B
:104680000E4C0A684B60551CA3420CD8002801D080
:104690004B600A600A4A136008680A4B186070BDD4
:1046A000581E821ADDE7084A30009B182A00EAE704
:1046B00000F00040E061FF1F140AFF1F40420F009E
:1046C000C8F00040CCF00040C0BDF0FF70B51F4CFA
:1046D00023793F2B01D93F2323711D4B22791A7077
:1046E0001878C0B207F044F918231A491A4A0B8007
:1046F0001A4913800B805380A379194980200B80BD
:104700000C21938001334B43164D191C0001834249
:1047100000D9011C2980D1806379002B11D101338C
:104720006371237A012B01D8022323726279237AE1
:104730000D4853430A21584307F05AFA0B4D28609D
:1047400070BDA02BEDD9A023EAE7C046D461FF1FBE
:10475000480AFF1FEE41FF1FBC43FF1FEC41FF1F34
:10476000EA41FF1FE841FF1F71020000C461FF1F03
:10477000F8B519210020FEF773FE114C011E114DF2
:1047800009D10C22104BC1CBC1C4280007F0A0FAFC
:10479000FFF79CFFF8BD0C2220000C49FEF734FE09
:1047A0000C2802D0084B43CB43C40C2228000849F4
:1047B000FEF72AFE0C28EBD00C220021E5E7C046CC
:1047C000D461FF1FA061FF1F68BE0011FC0C000038
:1047D000F50C0000F0B51D4C8022A5440400882093
:1047E00069465201400507F0EBF9902212016A4434
:1047F0001300200032C832C316C816C38023144CDD
:10480000144FA6689B033343A3603B6007F058F93D
:104810008823A0685B05C01806F0E2FF0025882306
:1048200029008022A0685B05C01840196944520025
:1048300007F0EEF880230135FF355B019D42EED194
:10484000A6603E60044B9D44F0BDC046FCEFFFFFF8
:104850002C43FF1F9808FF1F04100000F0B5040050
:1048600087B0002825D0684607F0BAF91B4C02280B
:1048700006D106226946200007F0AAF8002816D0C3
:104880006946002301250F262F00E25C0133100941
:104890001030874038002F00324097403A000243E2
:1048A0004A610439062BEFD16846FFF793FF07B042
:1048B000F0BD182269460A4807F082F96A46A3004B
:1048C000D358013305D01822FF21684607F000FABB
:1048D000EAE70134062CF1D1E9E7C0466509FF1F7C
:1048E00000090011F0B5002504000E0085B0AA42B1
:1048F00000D186E04B1C087801934B788978377992
:1049000009021943F3783F061B040B431F43039727
:1049100020706570252800D196E033D8112813D86F
:1049200006F0E6FE69002B012B012B012B01AA00EA
:10493000B800B1002B012B012B012B012B012B0106
:104940002B012B0105012501232800D1DEE0DB2806
:1049500000D034E1042A00D8ACE01025052A05D0A7
:10496000551F2A003800711D07F04AF80522310052
:10497000200007F045F82A003900601D07F040F8D4
:1049800005353EE0562859D010D8332800D19DE097
:10499000552839D02628DAD19F4B29001322180038
:1049A0001D0007F095F9FEF7A3FB5CE0712800D12C
:1049B00077E0722800D180E0602800D18BE0DC280D
:1049C000C5D1022A00D875E07378BFB26370B3789E
:1049D000A370032A05D0033A390092B2F01CFEF707
:1049E0004DFC10223900E01CFEF70EFDC51C00280E
:1049F00007DA60705CE00C222000884907F000F8BC
:104A00000C25280005B0F0BD013A854D0C2A13D8BD
:104A1000002A0AD02800019906F0F2FFFFF756FE9F
:104A20000C2228007F49FEF729FC29000C22601C7B
:104A300006F0E6FF0D25E4E70C22EBE7784D7A4B14
:104A40002A0043CB43C2E9E7013A734D0C2A11D83F
:104A5000002A08D00199280006F0D2FF0C22280075
:104A60007249FEF70BFC29001322601C06F0C8FFF8
:104A70001425C6E70C22EDE706226D49601C06F0FE
:104A8000BFFF0625BDE712226A49601C06F0B8FF89
:104A90001325B6E708226849601C06F0B1FF092516
:104AA000AFE77178F02905D8644B188801F0BAFD9A
:104AB0000225A6E7FF236370FAE7614B012A03D0C2
:104AC00072789A706270F3E79B78F4E72000FFF742
:104AD000A7FA050095E7013A594B5A4D072A10D815
:104AE000002A10D0012128005970019906F088FF92
:104AF00001F05CF829000722601C06F081FF082500
:104B00007FE70722EEE700225A70F3E7042A04D970
:104B10004D4D2F6006F0ACFEA860FFF797FD042214
:104B2000039003A9601C06F06BFF052569E7474D5C
:104B3000062A15D906222800019906F049FF002807
:104B40000ED006220199280006F05AFF062240499D
:104B50002800FEF793FB0123394A91780B439370A9
:104B600029000622601C06F04BFF072549E7012AB1
:104B7000A0D07078FFF772FE9AE7012800D0E6E631
:104B8000931E344F132B06D87378002B0BD100F0F3
:104B900015F900F04BF9304B39001D78601C6A1E86
:104BA00006F02EFF2DE7551E2A000199380006F069
:104BB00027FF38002949AAB2FEF760FBE9E7DA28A7
:104BC0001DD1042A00D875E7082A15D9B37972795E
:104BD0001B021343F27912041A43337A1B06134360
:104BE0003B603B68052231002000039306F008FF7C
:104BF0000422601D03A950E7FE236370F1E7DE285D
:104C000000D057E7511E012A01D10025F9E601988D
:104C100000F0B2FFF9E7C046A061FF1F74BE0011AB
:104C2000D461FF1FFC0C000068BE0011F50C0000F1
:104C3000AC61FF1F8C61FF1F3043FF1FF041FF1F5E
:104C4000D061FF1F8D42FF1FE061FF1F6509FF1F3D
:104C5000ADAC0000D163FF1FCF63FF1FAEDE0000CD
:104C600070477047020010B5094B0A32094C92B2E6
:104C7000DA815A8298811882207802F039FB042266
:104C8000054B012120781A7006F0B2FE10BDC04617
:104C9000BA42FF1F1A64FF1F1964FF1F013870B565
:104CA000042809D806F08CFD030928081200234BBC
:104CB0000221187806F09CFE70BD204B0821187860
:104CC00006F0A6FD00221E4B1A72F5E78022002492
:104CD0001B4B1A4D52001A8108211A682878DC7281
:104CE00006F0A6FE2100287806F07AFE012000F0EA
:104CF00063FE00F05BFFDFE7104B0821187806F039
:104D000087FD1048FFF72AF80F4B104A9B790020C7
:104D100093800F4A13808022094B5200D8721A8167
:104D200000F04AFE00F042FF0A4B9B78002BC3D0F4
:104D3000094A136006F01CFDBEE7C046F061FF1F84
:104D4000C461FF1FF941FF1FD461FF1FBC43FF1F58
:104D5000EA41FF1FD061FF1F34F0004010B5012968
:104D60000BD1012809D1054B1B78002B05D0262239
:104D7000034B04485A72FFF775FF10BDF263FF1F23
:104D8000C461FF1FC40900000300F0B50A4D8E186E
:104D9000B14202D152008018F0BD0C782F6824096E
:104DA0003C5D0F271C700C7801313C402F683C5D46
:104DB0005C700233ECE7C046E441FF1F0D22124B4A
:104DC00010B51A700C23114C11492370093A033B9A
:104DD0001048637006F014FE2D2301220E490F487F
:104DE000A371FFF7D1FF01220D49FFF7CDFF01228B
:104DF0000C49FFF7C9FF030000200B49020018709F
:104E0000FEF73CFA10BDC046EE63FF1FCF63FF1FE5
:104E10000BBE0011D163FF1F6709FF1FD663FF1F81
:104E20006609FF1F6509FF1FAEDE000070B5134C59
:104E3000142220001249FEF7E7FA431E114D132BEE
:104E400019D8AB78002B16D0431C2B7009236B703C
:104E500000230019037028780B4B01302900C0B2E1
:104E6000187006F045FF297822000139C9B20020E8
:104E700005F0DAFD70BDFFF7A1FFECE7D163FF1F7E
:104E8000AEDE0000CF63FF1FEE63FF1F10B5114BB6
:104E90001A781870002A0ED000280BD10E4B1A7801
:104EA000062A07D85423D340DB0703D50B4B1878C9
:104EB00002F01EFA10BD0028FCD0074B1B78012B16
:104EC00002D0033B022BF5D8044B0121187806F0E1
:104ED0008FFDEFE7F263FF1F1964FF1F1A64FF1FC6
:104EE00070B54A4E4A4A4B493070012005F028FC03
:104EF00000F0DAFEFEF7FCF806F002FF0322464956
:104F00004648FFF741FF2D24030004221C7044494A
:104F10000130FFF739FF30230470424D424C43709B
:104F200083702E3B062220004049EB87FEF76CFA87
:104F3000062813D0200006F053FE022809D00321D2
:104F4000200006F0F5FB8D23E3706E3B23711933CF
:104F50006371062220003549FEF790F9344B1B6837
:104F6000FC335C64FFF762FF0020FFF78FFF314CDA
:104F7000314A0121314B1278207802F07BF9304A16
:104F8000304B12780021207802F074F901222E4B68
:104F90001A702E4BDB78552B31D12D4B3B325A7288
:104FA0002C4B2D4AAB81EA812B826A8220213078FA
:104FB00006F09EFD0120404205F082FD01204042A6
:104FC00005F01EFEFFF7DCF8FEF790FE00F0B2FCE5
:104FD00001204042FEF766FF012006F011FEF0209E
:104FE00001F004FB0121307806F002FD307802F078
:104FF000DBFA1A4806F0A4FCFEF734FD70BD64220B
:10500000174B5B7953431A000A32CBE7F061FF1F5D
:10501000614C00115D4D00113043FF1F8C61FF1F7B
:10502000AC61FF1FBA42FF1F6509FF1FADAC000056
:105030004464FF1F1A64FF1F1842FF1FF941FF1F3E
:10504000EE63FF1FCF63FF1FC063FF1FD061FF1F11
:10505000C461FF1FC4090000CE090000F261FF1FF8
:10506000D461FF1FF8B50A0020230D001A40194231
:1050700063D05E4B1B78002B5CD0FFF7E7FA5C4BEC
:105080005C4C5D4E99686268737A8A1ADB039A42B7
:1050900002D36160FEF7E6FC327A217A531EDBB25E
:1050A000994205D1FFF72EF9002000F0B5FD15E07B
:1050B0009142F9D300272772FFF75EF9A37ABB422A
:1050C00002D0A772FEF754FD012000F0A5FD4B4F62
:1050D0003800FEF743FE390006F092FB637A002B9E
:1050E00025D0013BDBB26372002B20D1444BDB782F
:1050F000552B01D106F03CFBE37A002B12D00023A4
:10510000A27AE3729A4202D0A372FEF731FD3D4AC1
:105110003A4F1388380001331380FEF71FFE390021
:1051200006F06EFB642370795843FFF79BFD237AEA
:105130000133237220206840F8BD0BB2002B0ADA3D
:10514000314B187806F0B4FB002801D006F0A8FC1B
:1051500080200002EFE70224214206D0254B0120E7
:105160001A72FFF793FE2000E5E70B071ED5FFF745
:105170006DFA1F4B1F49204C98684A68637A821A5F
:10518000DB039A4202D34860FEF76CFCFFF7F4F8A9
:10519000FFF7B8F8012000F03FFD00F0E5FB2368C1
:1051A000DB0701D5FEF776FF0820C4E7CB0609D55B
:1051B000FEF7DEFC0D4B1B78002B01D1FEF7AAFD9C
:1051C0001020B8E70124214207D0104800F06CF805
:1051D00006F02EFD00F006FDC5E70424080020407F
:1051E0002142A9D0FEF77AFEBDE7C046F263FF1F59
:1051F000E061FF1FC461FF1FD461FF1FF941FF1F62
:10520000D061FF1FB861FF1FF061FF1FDC41FF1F6E
:10521000F0B51B4B1B4F1B883A8804001A4E1B4DE0
:1052200085B09A420DD832889A420AD3184B1A8810
:105230002B889A4205D1174A174B12881B889A422D
:105240001BD0052001F028FA3B8802AA138033887E
:10525000019053802B88114D93800F4B02A91B881E
:10526000D3800F4B2A78188802F044FF0D4B082199
:105270002878019A1C7006F0FBFC05B0F0BDC04612
:10528000BE63FF1FEE41FF1FEC41FF1FEA41FF1FFE
:10529000BC63FF1FBA63FF1FE841FF1F1A64FF1FB3
:1052A000F041FF1FB863FF1F13B50C4B1C78002C97
:1052B00011D1002801D00A4B18600A4A0A4B117814
:1052C0000A4A10780A4A01920A4A0092002205F01E
:1052D000A3FA200016BD1124FBE7C0461964FF1F86
:1052E000B463FF1F1864FF1F0864FF1F1A64FF1FC9
:1052F000F463FF1FF863FF1F10B5064B12201B78E5
:10530000052B06D1044B13221988044B187801F0A1
:105310009FFB10BD1964FF1FF041FF1F1A64FF1FA0
:1053200010B500240122114B52421870104B1C7012
:10533000104B1A8002F038F904220F4B21001A702A
:105340000E480C3206F0F4FA102221000C4806F048
:10535000EFFA07220B4B1C600B4B1C700B4B1C70A5
:105360000B4B1A700B4B1C7010BDC0461A64FF1F0C
:105370001964FF1FF041FF1F1864FF1F0864FF1F1F
:10538000F863FF1FF463FF1FCE63FF1FCD63FF1F92
:10539000F241FF1FCC63FF1FF8B5174C06002578BC
:1053A00006A814240078052D23D1B41F134FA5B2ED
:1053B0001824BD421DD88D1FADB2BD4219D8FA25A3
:1053C0006D00AA4215D21D000D4F0A3DADB2BD427F
:1053D0000FD80C4C26800C4C21800C4900240A80EC
:1053E0000B4A1380FFF714FF0A4B0421187806F0CC
:1053F0000FFA2000F8BDC0461964FF1F790C0000A9
:10540000750C0000EE41FF1FEC41FF1FEA41FF1F3A
:10541000E841FF1F1A64FF1FF0B50BB20D0089B001
:10542000002B00DB70E1A44E307806F041FA041E38
:1054300050D00378A22B00D122E1D02B1AD0912B8F
:1054400045D143780E2B42D19C4B82889A423ED163
:105450009B4A83681278052A39D1032018567F2881
:1054600035D0984B1B68002B31D05B68002B2ED0B9
:1054700098472CE08078072829D806F0A1F904285D
:10548000183F3F74A8D86378002B0CD101218C4BB6
:1054900019708D4B1A78002A5BD08C4B307801F054
:1054A000E9FE002855D00722854B1A7051E061783B
:1054B0000029F8D1E378002B11D0854A854B12786A
:1054C000307801F0D7FE60706378002BEBD12000BC
:1054D00006F0E6FA80200002684009B0F0BD784B83
:1054E0001B78022BF3D00121307806F0E1FA002876
:1054F000EAD10121307806F07BFAE5E76378002BEA
:10550000D1D16F4F032807D13B78052B02D101334E
:105510003B701EE00223FBE76F4B1A886F4B029330
:10552000002A0BD01B78002B03D00121307806F025
:105530009FFB3B78062B04D1013BE9E7029B1A70E5
:10554000F7E7042B41D10121029B3078197006F056
:105550004FFA5C4B1B68002BB9D01B68002BB6D0F0
:10556000574A107884E76378554F002B27D10622DD
:10557000211D5B4806F044FA62895A4B5A491A8049
:10558000A2895A4B1A80E3890B800521397058494A
:105590000A80584A1380228A574B1A80574B1B782F
:1055A000012B09D11F2001F077F8FA229200424323
:1055B0000421307806F05CFB0022484B75E7312B64
:1055C00000D070E70022454B1A700323A0E70622A3
:1055D0000021434806F0ACF90023454A042113801A
:1055E000444A30781380444A138006F011F90821A8
:1055F000307806F00DF9A379083B5A425341304AFE
:1056000003331370304B1B78002B06D0334B3078AC
:105610001A78002A06D001F06BFE0122314B52426B
:105620001A8096E70121197006F0E2F9F5E70821E2
:10563000307806F0EDF86378002B00D047E72C4B6C
:105640002D4F0293E388029A04211380294B30786E
:1056500003932389039A138063893B8006F028FA19
:10566000002800D033E7264B1B68002B00D12EE723
:10567000039902983A88098800881B68984726E7AA
:105680004379132B00D022E70389012B0AD11D4B4C
:105690001B78022B06D10821307806F0B9F8FFF705
:1056A0002BFE14E7052000F0F7FF082102003078F8
:1056B00006F0DEFA0BE7C0461A64FF1F051400006F
:1056C0001964FF1FB463FF1F1842FF1FF941FF1F3A
:1056D000EE63FF1FCF63FF1FF063FF1FF263FF1F27
:1056E000C163FF1FF041FF1FC863FF1FCA63FF1F95
:1056F000BE63FF1FBC63FF1FBA63FF1FC063FF1FB2
:10570000B063FF1FB863FF1F8020C001014200D0BB
:10571000E2E6CB0731D5324B1B78002B1DD0314E42
:1057200005AC3378052B1AD1023B23702E4B210098
:105730001B7823722D4B1B7863722D4B187801F068
:105740003DFD002809D007202A4B30701B68002B34
:1057500003D01B68002B00D098470120BCE60E2028
:10576000254B06221B7825492370254B1B78637037
:1057700002ABC01806F044F9D8E70223080018402D
:10578000194209D0174B1B78052B03D11D4B1888E4
:1057900006F0F6F902209FE60424214203D0FFF729
:1057A00037FD200098E6082308001840194200D170
:1057B00093E6154B1C78012C03D0022C0DD0082049
:1057C0008AE6124B124A134913481B88128809882B
:1057D00000880094FFF7E0FDF1E7FFF78DFDEEE7AD
:1057E000F263FF1F1964FF1FF241FF1FCC63FF1F0D
:1057F0001A64FF1FB463FF1FCE63FF1FF341FF1F37
:10580000CD63FF1FF041FF1FB863FF1FE841FF1F7B
:10581000EA41FF1FEC41FF1FEE41FF1F10B502A838
:1058200004880B20002C10D14968087849780902B7
:1058300001430C48814209D1022119800A4B598841
:105840001170DB7800205BB2537010BD074C0A204A
:10585000A142FAD102211980034B998811705B791A
:10586000F0E7C0466E2A0000B861FF1F6F2A0000F3
:10587000F7B5150008AA16884A680F4F14785278B1
:10588000120222430A24BA4214D10122DBB201924D
:1058900000962A0005F0C6FE041E0BD1074B1B68BC
:1058A000002B07D068782A7800021043424250410A
:1058B000013098472000FEBD022900002C64FF1F24
:1058C00030B5012503790400BFB02B4225D014491F
:1058D000408805F013FA28420CD0124B01A95B8DC9
:1058E00000220B8002234B800F4B5B888B806088EB
:1058F00002F0F6FA0D49608805F000FAC0070CD5F1
:105900000B4B01A91B8800220B8002234B80064B06
:105910009B888B80608802F0E3FA3FB030BDC046C0
:105920002464FF1F1C42FF1FB861FF1F1C64FF1F80
:105930007642FF1F10B5074C0749200005F094F987
:105940002000064905F090F90721054A054805F0B1
:105950004DF910BDFFFF00002464FF1F1C64FF1FF2
:1059600094BE00111C42FF1F10B5024803F03AF923
:1059700010BDC046C15800110221430888400B40A9
:105980000A31084003430E20024AD17881430B4379
:10599000D37070478D42FF1F064A1379410705D522
:1059A00080210B4380011371907170477F210B4060
:1059B000F8E7C0468D42FF1F054A5378002803D000
:1059C00080210B43537070477F210B40FAE7C0469C
:1059D0008D42FF1F0F21114BDA780A40DA705028F0
:1059E00010D901310A43DA702022D9780A43DA70DB
:1059F0004022D9780A43DA708022D97852420A4389
:105A0000DA7005E03C28EFD82828F1D81428F3D81C
:105A10000122D9780A43DA707047C0468D42FF1FD1
:105A2000F8B57F23324D04006E789E43314B984287
:105A300005DD76232B70363B33436B70F8BD2E4B60
:105A4000984203DA58232B701433F5E783B21A0017
:105A500000215F32294892B2294F297082422DD904
:105A6000A9708C4203DA5B421CB220232B700534F0
:105A700020B20A2106F0BCF804B2FA239B009C4233
:105A800033DB80232A785B4213432B706421200090
:105A900006F0AEF80A2100B205F0CAFE09B22A7873
:105AA0007B5C13432B700A21200006F0A1F80A2129
:105AB00000B205F0BDFE09B27B5C0AE08022AA704C
:105AC000002CDADA5B421CB220232B705F23092CF6
:105AD000E9DC1E430A2120006E7005F0A9FE09B220
:105AE000AA787B5C1343AB70A8E7632CCEDCEDE7B0
:105AF0008D42FF1F1B4E00001DFCFFFF2A08000007
:105B0000BEBE00117F23F7B5194FCD013E790400C9
:105B10009E433E71EDB2632806DD093B33433B7182
:105B200040231D437D71F7BD0300093304DA582378
:105B300033433B716C23F4E70E4B019300280BDADF
:105B40000423444224B23B710A21200005F070FE78
:105B5000019B09B25B5CE4E70928F5DD0A2106F048
:105B600047F8019B00B21B5C1E433E71ECE7C04648
:105B70008D42FF1FBEBE0011F8B50A4F05003B78ED
:105B80000E00002B0CD0084C2000FEF739FC33002F
:105B90002A0020003978FEF724FD2000FEF76EFC75
:105BA000F8BDC0463864FF1F9442FF1F70B50A4E0F
:105BB0000A4D07223100280005F00AFF002809D00D
:105BC000074C31000722280005F01AFF08212000A9
:105BD000FFF7D2FF70BDC0468D42FF1F3164FF1F2B
:105BE0003064FF1F7F2210B50A4B59789143033A66
:105BF0001A70103A0A435A7078220E219A70DA7895
:105C00008A43DA7006221A7139325A71FFF7CEFFD1
:105C100010BDC0468D42FF1F10B5002832D01E4C6B
:105C20000223E05E1D4B1B685B062CD50923322145
:105C3000584305F0DDFF4130FF3000B2FFF7F0FEC2
:105C40000520FFF799FE0422A35E154A63209342C4
:105C500005DC32331800642105F0CAFF00B20121CF
:105C6000FFF750FF207AFFF7B5FE0020FFF794FE04
:105C70000C4B1878053843425841C0B2FFF79CFEE0
:105C8000FFF794FF10BD0A21053005F0B1FF00B207
:105C9000FFF7C6FE0320D4E7B861FF1FD461FF1FE2
:105CA000DD2600001964FF1F70B50024094D28008F
:105CB000AC71FEF7A5FB10233E212800064AFEF733
:105CC00090FCA04200D13E34044B28001C70FEF72B
:105CD000D5FB70BD9442FF1FAEBE00113864FF1F9C
:105CE0000200F0B501270A480A4E51188B1A002B02
:105CF00000DCF0BD082415784308684038404000B7
:105D0000805B013C58406D08002CF5D10132EDE775
:105D1000FFFF0000CEBE0011F0B500250F269D420A
:105D200000DBF0BD4C5D070944403440A400A0589E
:105D300001357840F3E70000F0B589B06A460D0000
:105D40000B000F27110010351C78013326002409A1
:105D50003E40167054700232AB42F5D12023024A05
:105D6000FFF7DAFF09B0F0BDD4BE0011F0B54E78F0
:105D70000B7889B036020C00170001901E43012AEF
:105D800061D9954B9E4200D877E001339E421CD1E9
:105D9000062A17D1CA788B7812021A430B791B0492
:105DA00013434A7912061A438C4B5A6100221A7027
:105DB0005A808B4A5A608B4A9A608B4ADA6000207C
:105DC00009B0F0BD88225205EEE7884B9E423CD1D7
:105DD00082498B78002B00D0F6E00C2A31D10F22BB
:105DE000A3789343E27812021343227912041343F7
:105DF0006279120613434B60E279A07912020243E2
:105E0000207A00041043627A12060243CA60E27AE2
:105E1000A07A1202024376484A81834208D80423BA
:105E20006E49142201980B7005F0EAFD1420C7E7B3
:105E30001201D21889235B059A42F0D801238B7096
:105E4000BDE7022AFAD00523EAE76A4A012396420F
:105E5000E6D1FFF751FA052F0CD9E378A2781B029F
:105E60001343227912041A4363791B061343624ACF
:105E70000393136005F07CFCA1E7584D2B78002BB1
:105E80009DD1AB78002B00D1A0E02B8901339BB2D0
:105E90000093B34200D091E0132AD4D9CF7C8B7CFD
:105EA0003F02122120001F43FFF71AFF874200D054
:105EB0008EE0002E3DD1E378A2781B0213432279B5
:105EC000E96812041A4363791B06134303930A22F9
:105ED0008B4212D1FF23A370E370237163716B892E
:105EE000002B09D1E37B227C1B0212041343A27B0B
:105EF00013431B0901336B8100226B89002B8ED069
:105F0000002A67D1686837013818000B6B690003F5
:105F10000390984205D9686105F062FCEB78013383
:105F2000EB7068681022A11C381805F071FD2E81F5
:105F300045E76F89009A7B1E9BB293423AD1E27883
:105F4000A37812021A43237905A81B04134362792C
:105F50006C6812061A43EB6800920392211D0C2212
:105F6000049305F04DFD0120260004A9404210369F
:105F7000FFF7E2FE013F012F17D1009A0B232861A2
:105F8000824200D04CE704221C49200005F040FD6D
:105F9000042203A9686805F013FEE968039AFF2349
:105FA000914200D13CE7F73B3AE73100FFF7C4FEEE
:105FB0001036DFE70923B742A4D831E7009BB3428C
:105FC00000D9FCE607232BE7022329E7032327E771
:105FD000062325E70A2323E7FFFE00009C42FF1F5C
:105FE00000000111FFFF00005048593601FF00007A
:105FF000FFFF001102FF000034F00040A842FF1F25
:1060000010B5034C0B000122210000F06BFA10BD0B
:10601000C16100110B8870B506000D000224162B1B
:1060200011D92B000322094900F05CFA041E0AD1A1
:10603000074B2A881B88191C934200D9111C300079
:1060400089B200F0EFFA200070BDC046ED6100118A
:106050004A64FF1F10B54A780400013A0B00022081
:10606000012A07D80A78002A04D005222000024914
:1060700000F038FA10BDC0461B6200110A7810B556
:106080000B0004000220002A04D00722200002494D
:1060900000F028FA10BDC046C76200110A7810B59A
:1060A0000B0004000220002A04D00922200002492B
:1060B00000F018FA10BDC0462D63001110B5034C56
:1060C0000B000B22210000F00DFA10BD5D630011E2
:1060D00010B5034C0B000D22210000F003FA10BD97
:1060E000CF63001110B5034C0B000F22210000F00C
:1060F000F9F910BD296400110A7810B50B000400ED
:106100000220002A04D011222000024900F0EAF9FE
:1061100010BDC04639640011002310B513221900C8
:1061200000F0E0F910BD000010B5034C0B00172281
:10613000210000F0D7F910BD8B640011002310B5C9
:106140001922190000F0CEF910BD000010B5034C63
:106150000B001B22210000F0C5F910BDC564001121
:10616000F7B584890D0006000121002C22D0002300
:106170008268D3561778002B1EDA0C2C1AD90C3CE7
:10618000A4B2131940880093230002F086FE431E38
:10619000984101307B06DB0F6B703F23013C1F40B1
:1061A000A4B22870AF70AC80002C07D0B368013364
:1061B000AB6000210800FEBD0020EBE7AC60F8E713
:1061C0000B7803704B8843704B881B0A83700B79E4
:1061D000C370042070470420022B06D1002053789E
:1061E00011781B02009A0B43138070470B880370D1
:1061F0000B881B0A437002207047042000998342D9
:106200000AD1537810781B0203430B80D37890781F
:106210001B02034300204B807047F8B50D004B78FC
:1062200001240021461C03702B788B4201D82000EA
:10623000F8BD6B78B01C4F1C012B10D18900691878
:106240004B88022233704B88B9001B0A737069189F
:1062500005F0BEFA04360434A4B2F9B2E4E712231E
:1062600059436B185A88043132705B8810221B0A1C
:106270007370691805F0ACFA12361234ECE770B599
:10628000049D14001E00052B01D8042070BD637806
:1062900012781B0213432B80E378A2781B0213436E
:1062A00002226B802A71211D681D063E05F090FABE
:1062B000B2B22A81E92AE8D82800A11D0A3005F0E7
:1062C00087FA0020E2E7002310B50A789A4201D845
:1062D000900010BD9A008A185488013304705488C5
:1062E000DBB2240A4470948884709288120AC270C7
:1062F0000430EAE710B51100029C062B04D00420FC
:106300001022142B01D010BD022222714B78087884
:106310001B0203432380CB7888781B0203436380EE
:106320000431601D05F054FA0020ECE710B50C783C
:106330008B7804315C43E4B203702200013005F035
:1063400047FA601C10BD0420022B06D100205378B0
:1063500011781B02009A0B431380704710B50C0094
:106360000A88023105F034FA208810BD70B50400A7
:106370000D0004981100012B01D8042070BD16787F
:1063800052781202324302800200F13255701470CA
:10639000E125002C00D10C35023B9AB24280AA4282
:1063A000EBD80231043005F013FA0020E6E70420B0
:1063B000009983420AD1537810781B0203430B8063
:1063C000D37890781B02034300204B80704710B5B0
:1063D0000C000A88023105F0FBF9208810BD00008E
:1063E00070B501211E000420049C0E400B4218D100
:1063F000CB40DDB28D4214D90A49DBB209889942FB
:106400000FD32300EE331D70330058001118497864
:10641000165C0902314301332152D9B28D42F4D8BE
:10642000002070BDB442FF1F10B50C000A88023175
:1064300005F0CEF9208810BD10B50C788B780431AA
:106440005C43E4B203702200013005F0C1F9601C26
:1064500010BD10B511000298032B01D8042010BD07
:1064600014785278043B120222430280CA788C7856
:106470001202224342809AB28280EB2AEED8043183
:10648000063005F0A5F90020E9E710B50C000B88EF
:1064900003700B881B0A43704B8883704B881B0A60
:1064A000C3708A880430063105F092F9A088043060
:1064B00080B210BD0420012B03D100201378009A74
:1064C0001370704710B50C000B8803700B881B0A03
:1064D00043704A880230043105F07AF9608802304E
:1064E00080B210BDF0B589B003931E4B02924200FA
:1064F0000700D05A019102F020F81325061E2DD076
:10650000029B01240370019B002B04D00019039906
:106510009847001984B26B461B7A5BB2002B0FDAE6
:106520001021380002F01CFB1925002813D130007F
:106530003219E1B202F066FC051E0CD10C34A4B293
:10654000042304AA380005A993800696948101F0DB
:10655000AFFD051E02D0300005F0D2FA280009B0C8
:10656000F0BDC0464864FF1F70B505000C00002850
:106570000CD00020814209D010222000044905F0EF
:1065800027F901202B7823736B78637370BDC046A5
:1065900014BF0011F0B506000D0017001C0085B0F7
:1065A00002291BD00020102907D1022B07D0102B65
:1065B00003D115E00020102C08D005B0F0BD6946CD
:1065C0003800FFF7D1FF2A0069460BE0694630002A
:1065D000FFF7CAFF22006946380004E0022BE9D128
:1065E0002A003900300005F093FBE6E7031CF02891
:1065F00000D9F023032008499AB2013A0B80D3173F
:10660000034006499B189B100B80D30F04499B182D
:106610005B100B807047C046B842FF1FB642FF1F99
:10662000B442FF1F034B1B888B4202D3024B400036
:10663000C1527047B842FF1F4864FF1F014B400022
:10664000185A70474864FF1F1722014B1A80704781
:106650004864FF1F70B505000E2005F0D9FA041E2E
:1066600013D0D0230370002306228370074945709E
:10667000033005F0ADF8064B2100DA8A62811B7EFB
:106680002373044B187805F0FBFA70BD6464FF1F98
:106690005464FF1F0843FF1F262803D8024B400005
:1066A000C05A70470148FCE7BA42FF1FFFFF0000D5
:1066B00070B506000C00094D1C220021280005F0D1
:1066C00037F9074B1E70074B1C7005F039FB01238F
:1066D000002801D0002312202B7070BD5464FF1FCE
:1066E0000843FF1F7564FF1F70B505000D4C0800BF
:1066F000E260A16010220021656005F059F90128CF
:1067000003D11021A06802F058FD102200212800BA
:1067100005F04EF9012803D11021606802F04DFD0B
:1067200070BDC0465464FF1F70B5041E05D100291A
:1067300003D006220D4805F04BF80D4B1D78012DB6
:1067400011D1002C05D102221A7005F0E1F82800C1
:1067500070BD00221A70074B1B78FF2BF7D020006A
:10676000FFF778FFF3E70025F1E7C0466464FF1FF9
:106770005464FF1F0843FF1F030010B5002801D118
:10678000002010BD00780B4A002803D15988D1821F
:106790001B7913761378022BF2D10023984200D193
:1067A00003331370044B1B78FF2B01D0FFF752FF0C
:1067B0000120E6E75464FF1F0843FF1F002911D0A2
:1067C00000280CD04B79012803D1402252421343B8
:1067D00003E03F221340032802D001204B71704791
:1067E0004022F4E70800FAE770B5094D0100287867
:1067F00000280BD0074C0622200004F0E9FF2100FE
:106800002878FFF7DBFF200005F0E2F970BDC046F5
:106810007464FF1F4E64FF1F00290AD0012808D1AD
:106820003F224B799343C02B03D0403B5A42534104
:10683000981C704770B5174D06002B78FF2B15D0AC
:106840000A2005F0E5F9041E10D0D0230370C83BE0
:106850008370114B11491B784670C37006220430B7
:1068600004F0B6FF2100287805F00AFA0C4B1B78DB
:10687000012B0DD10B4B1B68002B03D09B68002B09
:1068800000D09847084B04211878084A05F0D0F842
:1068900070BDC0460843FF1F7464FF1F4E64FF1F96
:1068A0007064FF1F9C64FF1FA064FF1F60EA00006C
:1068B000014B98687047C0465464FF1F014BDB686A
:1068C000186870475464FF1F074B10B5DA681368E7
:1068D00001331360054B1878FF2803D08021C901CC
:1068E00005F086F810BDC0465464FF1F0843FF1F23
:1068F000F7B50E0002F0C8F8051E1CD00E4B06625C
:106900001F78002F00D10778AB791020019305F094
:106910007FF9041E0FD0D0230380C73B8370019BF7
:10692000E91DC3700622043004F052FF2100380034
:10693000E66005F0A5F9F7BD0643FF1F014B187887
:106940007047C0467464FF1F054B002805D1054BF6
:106950001A78054B002A00D1014B18007047C04639
:106960006464FF1F7464FF1F4E64FF1F014B58686F
:106970007047C0465464FF1F024B1868431E98417D
:10698000C0B270477864FF1F421E03000120152A21
:1069900003D9FF3B5A425341D8B27047F0B51C00AF
:1069A00000230E0085B0039002920B70029A93426E
:1069B00001D3002019E0E55C5A1CD2B2002DF8D0BA
:1069C000029851198142F4DC0233DFB2A35C180053
:1069D0000193FFF7D9FF002807D0013D019A0399E1
:1069E000EBB233708A4202D1E01905B0F0BDDB1979
:1069F000DBB2DBE710B50C0002F09EF803001220BA
:106A0000002B03D02100588805F092F910BD00003A
:106A100070B50E4D84006359002B15D0186A0028FC
:106A200001D004F07DFF2B59586A002801D004F0F2
:106A300077FF2B59986A002801D004F071FF28597C
:106A400004F06EFF00232B5170BDC0468464FF1F0D
:106A50001C4B70B504000E00150099420AD11A4B68
:106A60001B68002B01D1122070BD1B68002BFAD0CF
:106A70009847F9E7154B994215D1134B1B68002B2A
:106A80000AD01B68002B07D09847002804D1104B70
:106A90001C70104B1D70E7E729002000FFF7AAFFCC
:106AA0000028E1D1F3E7080001F0EEFF0028DAD07A
:106AB00003780320A342D7D12900300005F038F92C
:106AC000D2E7C046FEFF00008064FF1FFFFF00000A
:106AD0007D64FF1F7C64FF1FF7B50400808801F010
:106AE000D3FF0025A84203D00578A08802F008F85B
:106AF0001C4E3378002B1FD0AB421DD11A4B2800FF
:106B00001978FFF777FF002818D000233370A37996
:106B10000820A778A688019305F07AF8011E0DD009
:106B2000D0230370CA3B8370019B477086808371BA
:106B3000280005F0A5F801E0002DE8D1A0880B4B56
:106B40008200D358002B01D0FFF762FF1721A088E5
:106B5000FFF768FDA08801F027FDA08801F0FEFD89
:106B6000F7BDC0467D64FF1F7C64FF1F8464FF1F68
:106B7000F0B587B01D000CAB1B88070001930DAB6F
:106B80001B88142002930EAB1B88160003930FABD7
:106B90001B880091049310AB1B88059305F038F80F
:106BA000041E1AD0D0230370CB3B47708370C6708D
:106BB000062229000430002D11D004F009FE019BAB
:106BC00021006381029B0098A381039BE381049BC6
:106BD0002382059BA37405F053F807B0F0BD04F0C1
:106BE000A7FEECE7F7B5009308AB1B8807000C2065
:106BF0000D001600019305F00BF8041E13D02800B9
:106C000001F042FF00280FD00078D0232370C93B49
:106C1000A370009B21002381019B6770A580E68003
:106C2000638105F02DF8F7BD014B1878EDE7C046FC
:106C30000843FF1F13B5040064890389C288818853
:106C4000C0780094FFF7CEFF13BD000010B5044CD0
:106C50002068002803D004F063FE0023236010BDE9
:106C60008864FF1FA122F0B5818892004A43384B07
:106C7000384F1B6804009B189D2292009B18827954
:106C800089B01A603B68002B5FD01D78324B1B68BF
:106C9000002B04D05B68002B01D000209847260011
:106CA00008363100E079FFF7B7FD237DE07102007F
:106CB000E0780493638A29000393238A0293E3898B
:106CC0000193A38800933300FFF752FFE378002B72
:106CD0000BD1E289A379A18802920196E27928007A
:106CE0000092012201F0DAFEE0703B68002B20D018
:106CF000FFF7ACFF194D287800281AD0184B1978E7
:106D0000FFF778FE002814D02B78E6780820079348
:106D1000A78804F07DFF011E09D0D0230370CA3B71
:106D20004670837087808671079804F0A9FF00235E
:106D30002B701721A088FFF775FCA08801F034FCA8
:106D4000A08801F00BFD09B0F0BD064B9DE7C046E1
:106D50003409FF1F8864FF1F9C64FF1F7D64FF1FB1
:106D60007C64FF1F0843FF1FF8B5070008000E00F2
:106D700001F08AFE041E18D02620FFF78DFC051EA8
:106D800000D12578062004F043FF041E0DD0002119
:106D9000062204F0CDFDD0232370C23B2100677092
:106DA000A370A680E8B204F06BFFF8BDF0B585B023
:106DB00001930AAB1B78070002930BAB1B7808000A
:106DC0000D000092039301F05FFE061E22D01020FA
:106DD00004F01EFF041E1DD01022002104F0A8FDA7
:106DE0002620FFF759FC002800D13078D0232370EB
:106DF000C13BA370009B21002372019B67706372EB
:106E0000029BA580A372039BC0B2E3720C9BE3605C
:106E100004F036FF05B0F0BDF7B50D00019001F0AC
:106E200033FE071E20D00E2004F0F2FE041E1BD0FD
:106E30002620FFF731FC061E00D13E78D0232380A8
:106E4000C53B0622A370F91DE01C04F0C1FC019BA8
:106E50002A0063810123DD401A401D402100227376
:106E60006573F0B204F00CFFF7BD0000F0B585B01B
:106E7000029010000D0017000A9E039301F004FE1B
:106E8000041E31D0029B002B2ED1039B02795B079D
:106E900024D5122313430422002E08D10B99002974
:106EA00005D10C99002902D10D9900291AD01A4355
:106EB0000D9B2271002B00D0C9E0002E00D1CFE045
:106EC000002D00D0CCE0606A002801D004F028FD3D
:106ED0001C21300004F0F4FC606205E002239A43B8
:106EE0000E33D7E793432371654BBA00D458002C77
:106EF00000D1AAE0002E10D0236A002B03D11C2061
:106F000004F04EFC20625E4BBA00D358186A002889
:106F100003D01C22310004F05BFC0C9B002B12D030
:106F2000574CBB001D596B6A002B03D1162004F08F
:106F300037FC6862BB00E358586A002803D0162269
:106F40000C9904F045FC0D9B002B11D04C4DBC005E
:106F50006659B36A002B03D1142004F021FCB062FF
:106F60002B59986A002803D014220D9904F030FCA4
:106F7000380001F089FD051E67D0414BBA00D35897
:106F8000002B62D01A6A3420002A00D11C389A6A79
:106F9000002A01D0143080B20B9A002A01D01C3094
:106FA00080B25B6A002B01D0163080B204F030FE54
:106FB000041E4AD01822002104F0BAFC2620FFF754
:106FC0006BFB0190002801D12B780193D023237013
:106FD000029B200063700A23294EA370039BBD000F
:106FE000A371AB59A780196A1830002905D01C225B
:106FF000A06004F0EDFB200034307359996A002939
:1070000007D0030014221433E060029304F0E0FB85
:1070100002980B9B002B08D003001C221C330B99F9
:107020002061029304F0D4FB02987359596A002935
:1070300003D01622606104F0CBFB6B462100187967
:1070400004F01EFE3800FFF7E3FC05B0F0BD10228F
:107050000D9B0D991B69A018236204F0B9FB2CE766
:107060000B9B002B00D13FE7012D00D03CE7606A6D
:10707000002801D004F054FC1C210B982AE7C046DC
:107080008464FF1F10B5044C2068002803D004F06E
:1070900047FC0023236010BD7864FF1F0B4B07B52E
:1070A0001A68002A01D100200EBD6946531C012038
:1070B00012780731FFF772FC0028F4D00278012320
:1070C000100018401A42EED0EEE7C0469464FF1F4D
:1070D000F0B51F4F01203B6887B0002B25D09B786F
:1070E000059300F0B3FB002821D00A20FFF7D4FA63
:1070F00004000B20FFF7D0FA164B05001E78731E14
:107100009E413B68F6B2191DD878FFF757FB3B68E4
:107110002900DA7A043303929A790193029200905B
:1071200033002000059A04F08BFD07B0F0BDFFF797
:10713000B5FF002805D00620FFF7AEFA04000720AF
:10714000D8E70820FFF7A8FA04000920D2E7C046D4
:107150007864FF1F7464FF1F70B50A4E0400337813
:107160000D00FF2B0DD0042004F052FD011E08D0AD
:10717000D0230370CE3B45708370C470307804F028
:107180007FFD70BD1843FF1F70B5040006200D0081
:1071900004F03EFD011E0AD0D0230370CD3B837066
:1071A000054B44701B688580187804F069FD002C3D
:1071B00001D0FFF767FF70BD7864FF1FF8B5264F59
:1071C00006003B680D001124002B05D10522234B3E
:1071D0001B78134202D112242000F8BD204A10244B
:1071E0001268002AF8D01278002AF5D0DB0719D5EA
:1071F0002B789A1E012A1AD80C2004F0D1FA1324F5
:1072000038600028E8D000230A2243702900067065
:10721000023004F0DDFAFFF75BFF041E0AD0FFF72F
:1072200031FFD9E700F012FB0028E1D1E4E7002BA1
:10723000E2D0D0E70B4B1B78032BCDD11D20FFF7FD
:107240002BFA094B18800028C6D0084B0421187867
:10725000074A04F0EDFBBFE77864FF1F7564FF1F6A
:107260009464FF1F7464FF1F7264FF1FA064FF1FFC
:1072700060EA0000F7B50193194B14001A78052352
:1072800006000F0012201A4221D0012920D1154BEF
:107290001D68002D1BD002201F2C18D8002C02D0F6
:1072A000019B002B13D0104B1F221E706E1C00215F
:1072B000300004F03DFB01992200300004F088FA10
:1072C000310020002C70002F06D004F0B9FAFEBD6A
:1072D000064B12201D68DCE704F00AFDF7E7C04604
:1072E0007564FF1F9464FF1F1843FF1F9064FF1F06
:1072F000F8B50F4E12243368002B17D01B780F3CC3
:10730000834213D100250B4F0221387804F080FA14
:10731000094B042138781D8004F07AFA074B2800C5
:107320001D8033685C7004F07BFC04002000F8BD15
:107330007864FF1FA064FF1F8C64FF1F7264FF1F2F
:1073400070B5012823D11B4C2388002B03D01A4A87
:107350001578002D07D0194B1B68002B02D0187828
:10736000FFF7C6FF70BD3B2B02D93C3B2380F9E7FA
:10737000134E0221307804F04BFAFA22238892004F
:1073800002215A43307804F073FC2580EAE70B4B66
:107390001B68002BE6D00B4B1B785B07E2D5084B34
:1073A0000221187804F034FA0022024B1A80FFF709
:1073B00069FED7E78C64FF1F7064FF1F7864FF1FAE
:1073C000A064FF1F7564FF1FF8B51E4D28680028D4
:1073D00003D004F0A5FA00232B601B4E3068002870
:1073E00003D004F09DFA00233360184F05243B7846
:1073F00018002040234221D0154800F02BFA3B789A
:10740000234213D0202004F0CBF92860002813D0A9
:107410002022002104F08CFA202004F0C1F9041E7F
:10742000306005D02022002104F082FA002004E020
:10743000286804F075FA2C601320F8BD00F00AFAF1
:10744000F4E7C0469464FF1F9064FF1F7564FF1F3C
:107450000C43FF1F10B50A4C23681A1E0ED00028DB
:1074600008D10130587004F0DBFB002805D02368F8
:10747000002B02D00021FFF787FE0122100010BD73
:107480007864FF1FF7B5274E050033680191181E79
:1074900021D05C78244F012C30D1FFF7FFFD00286C
:1074A00025D02000FFF7F8F80400412814D91F4B1D
:1074B000022118781E4A04F0BBFA1E4B3C3C1C808B
:1074C000022233685A703B78002B14D128000199AE
:1074D000FFF75AFE0120FEBDFA2292004243002A25
:1074E000EED0124B0221187804F0C2FBE8E7FFF758
:1074F000D3F80200F3E700233B70EBE73B78002B67
:10750000E8D1032004F084FB011E08D0D0230370CF
:10751000CC3B457083703368187804F0B1FBFFF7FB
:10752000B1FDD7E77864FF1F7064FF1FA064FF1FE1
:1075300060EA00008C64FF1F10B5174983880200C1
:107540008B4220D011D815498B4217D01449002006
:107550005B1899B2012907D8926811785A425341B1
:10756000D8B2FFF7F9FD012010BD0E4A00209B188C
:1075700007229BB29A424041C0B2F5E7836818786F
:10758000FFF768FFF0E7836899785A78090218785E
:107590001143FFF777FFE7E70A200000062000000D
:1075A000F8DFFFFFAFDFFFFF014B18707047C046E9
:1075B0001943FF1F10B5064C207001F041FA2078E6
:1075C00004F07EFB0521207800F062FD10BDC0466E
:1075D000A064FF1F0BB273B50D00002B00DBC4E0ED
:1075E000884B187804F064F9041E0ED00378912BB0
:1075F0000FD0A22B00D1A1E0834B1878FF2852D0E6
:10760000210004F03DFB00284DD18020000268409D
:1076100076BD43780F2B76D013D8052B70D00E2B68
:10762000EAD18088794B98422BD8794B98421BD865
:10763000784B9842E0D1A3681878591CFFF774F88A
:1076400038E03E2BD8D18378032B74D06CD8012B33
:107650006ED0022BD0D1704B1B68002B23D05B68FF
:10766000002B20D098471EE06C4BC0180C28C3D8C4
:1076700004F00EFB1DC2C2150BC20B0B0B3223C252
:107680003C00674BC0180728B6D8664B1B68002B18
:1076900009D01B68002B06D0200098470AE0A36899
:1076A0001878FFF7C7F8200004F0FAF9ADE7A068F2
:1076B000FFF762F800289FD0F5E7A3681B78002B3E
:1076C000F1D0554B1B68002BEDD01B68002BEAD086
:1076D000210055489847EDE74F4B1B68002BE2D03F
:1076E0001B68002BDFD021005048F3E7504B1B688C
:1076F000002BD8D05B68002BD5D021004348E9E7A8
:10770000FFF7EAF9CFE780884A4B984203D04A4B0B
:10771000984200D070E7464B1B68002BC3D05B68D3
:10772000002BC0D02100D5E7153B012BBBD963E767
:10773000FFF798FAB7E7FFF77DFAB4E73F4B1B78FE
:10774000042B07D100236A4613800179408800F09A
:10775000C5FCA8E7364B1B68002BA4D05B68002B48
:10776000A1D00100364898479DE7012421420AD064
:10777000294B1B68002B04D05B68002B01D0002034
:107780009847012043E78B070AD5264B1B68002B3F
:1077900004D05B68002B01D020009847022036E718
:1077A0000421280008400D4200D131E7254E3388DE
:1077B000002B21D0013B9BB23380002B1AD1FFF765
:1077C000DBF800280AD0204B1C70164B1B68002BDE
:1077D00004D05B68002B01D020009847FFF7C6F863
:1077E000694601F001FD6846FEF7FEFF1D20FEF729
:1077F00053FF308004200AE7024B187804F008F8A1
:10780000F8E7C046A064FF1F1943FF1F0E200000C9
:1078100001200000091000009864FF1FFEDFFFFF39
:10782000AFDFFFFF9C64FF1F0C2000000B20000057
:107830008064FF1F0D200000132000007564FF1FEF
:10784000FFFF00007264FF1F7064FF1F10B501F09E
:107850009BF910BD014B18607047C0469C64FF1F28
:107860000B880020162B01D817230420014A13800F
:107870007047C0464A64FF1F00207047074A030054
:107880001188814207D091880020994202D10130AD
:107890008000101870470020FAE7C046A864FF1F58
:1078A000F0B58F7806000D00C5B01E2F15D1FFF77B
:1078B000E5FF051E03D10024200045B0F0BD0022E5
:1078C0003B003100C078009200F0B2FB0400A81C1D
:1078D00000F0D2FBFF23EB70EEE7264B0624039368
:1078E0001B78FF2BE8D0182FE6D87B08224A013BF3
:1078F000DB0002929A589446002ADDD0029AD318EF
:107900005B68002BD8D00878002802D14B78012B77
:1079100002D10624122FCFD107AFAB886978009728
:107920006446AA68A047041EC6D1AB78029A5B08D9
:10793000013BDB00D318390030005B689847041E18
:107940000BD1AB78042BB6D0039A3100107822000B
:10795000009700F06DFB0400AEE76A78002AABD117
:10796000AA7805A93B88087130000A704B80FEF7A1
:1079700047FBA0E71C43FF1F24BF00111D4B37B579
:10798000050098420BD000290AD1FFF777FF0028A5
:1079900005D11948FFF772FF002800D0058037BDD8
:1079A00001291AD1FFF76AFF041EF8D001235B42B8
:1079B0000380A378FF2BF2D0FE2B07D00023E078C2
:1079C0001422009329001E3300F032FBA01C00F0AB
:1079D00053FB01235B426380E1E70229DFD10139D8
:1079E00001F0BEF80028DAD12800FFF747FF041E97
:1079F000DFD1D4E7FEFF0000FFFF0000022210B538
:107A0000074B52421A80074801325A809A80DA8026
:107A100000F07EFA044801F025F8002010BDC046B1
:107A2000A864FF1FA17800117D7900110388F7B5C4
:107A30000400002B02D102252800FEBD426802216D
:107A4000137825485268FEF7A5FD00282ED0234F55
:107A500001253A88002AEFD0802321885B02012586
:107A60009B1A9942E8DC0C2003F09AFE061E31D0E6
:107A70003B8822889C4600231800019561469DB2F0
:107A8000491989B2AA421BD8002801D062443A8021
:107A900000233000082208C0210003F099FE104A9C
:107AA0001368002B13D100251660C5E76268022118
:107AB00013780C485268FEF76DFD0028C7D1BAE76D
:107AC00060681D014019418101330198D6E71A0011
:107AD0001B68E6E71325AFE792BF00111A43FF1FAB
:107AE000A464FF1F90BF0011014B18707047C0467F
:107AF0001C43FF1F14230A0010B51A40194204D07A
:107B00000122102101F048F810BD4B06F9D40120E4
:107B100088434000F8E710B514008B0604D5012215
:107B2000102101F039F810BD08230A001A4019424B
:107B300002D14BB2002B0FDA102101F02DF80028F2
:107B400008D02300F2331B78002BECD0F1342378DB
:107B5000012BE8D10020E6E703208907FAD4E2E709
:107B6000F0B51F00184B85B01C680190029103927C
:107B7000002C27D1200005B0F0BDA5683301ED1819
:107B80006B89019A934211D3029A93420ED8002F27
:107B900004D10A9B002B10D12C00EBE73B00297885
:107BA000039A6868FEF7F6FC0028F2D10136B6B2F7
:107BB000A388B342E1D82468DAE7A3680A9A5B890C
:107BC0001380E9E70026F3E7A464FF1F37B50C0034
:107BD0000A8849880123914217D3002A15D0651DD0
:107BE00023792A0002210A48FEF7D4FC102300283A
:107BF0000BD023796188208800242A000094FFF7A5
:107C0000AFFF0A23A04200D0230018003EBDC046AB
:107C100092BF001113B50A000888498801238842E1
:107C20000BD8002809D00024137905320094FFF7FF
:107C300097FF0A23A04200D02300180016BD13B5F9
:107C40000A0008884988012388420BD8002809D0F7
:107C50000024137905320094FFF782FF0A23A04223
:107C600000D02300180016BDF0B58BB003904A88F1
:107C700008880E000123824255D3002853D00023E8
:107C8000012704AC23700022718813000092FFF7D3
:107C900067FF051E3ED02078002835D12B78022BB7
:107CA00018D167706A8983000130E31880005A8018
:107CB00069680222201803F08BFD23780133DBB2C0
:107CC0002370042B19D93B006889013080B2002B46
:107CD000D9D01FE002236370122358436A89231806
:107CE00004305A8069681022201803F071FD23784F
:107CF0000133DBB22370002BE5D10C4A6B899B1852
:107D00005A425341DBB2DFE76378012BE4D12B7891
:107D1000022BC7D022780A23002A04D0210003981E
:107D2000FEF798F9002318000BB0F0BD0100FFFF2B
:107D30000F4BF0B504001868002816D083685D89E1
:107D4000A54207D88288AE18B44203DA12019A1805
:107D5000934201D10068EFE71E005F891036A74209
:107D600004D1002900D00D801800F0BD3300EFE7EA
:107D7000A464FF1F70B505000C0008880021FFF700
:107D8000D7FF03000120002B04D022002800197A1D
:107D9000FFF7C1FE70BDF7B50C0000250190230070
:107DA000EE331B78AB4201D800200AE06B00E65AA4
:107DB00000213000E718FFF7BBFF002802D1268022
:107DC0000130FEBD017A0198FFF794FE002802D031
:107DD0003B882380F5E70135EDB2E0E710B50400FC
:107DE00008880021FFF7A4FF03000120002B03D027
:107DF0002000197AFFF77EFE10BD0000054B1B68BE
:107E0000002B01D1180004E09A6852898242F6D111
:107E100098887047A464FF1FF0B50E27002687B02E
:107E2000039302ABFF183E8005001F4B40891400EE
:107E3000984207D02B78013000976A6880B2FFF72C
:107E40008FFE060002212B7818486A68FEF7A2FB15
:107E500000280FD06C892000FFF7D0FF002802D047
:107E6000013C0419A4B2039B002B00D01C803000FD
:107E700007B0F0BD02212B780D486A68FEF78AFB37
:107E80000028E7D102212B780A486A68FEF782FBB6
:107E9000002807D0002EDED03B88A342DBD17489B6
:107EA000013CDFE76C89DEE7FFFF000092BF0011B5
:107EB00090BF00118EBF001110B50C00FFF7DEFC63
:107EC00003000220002B0AD0002C00D023609B78F6
:107ED0001720FE2B03D00138FF2B00D1002010BD4E
:107EE00073B50D0001A904001600FFF7E5FF172880
:107EF00005D0002E04D129002000FEF727F976BD19
:107F000001221021200000F047FE0028F3D0F6E700
:107F1000014B18607047C046B464FF1F37B56B460D
:107F20009D1D010004000222280003F069FD2B883A
:107F3000B02B0ED12379122B09D12300FA331B78F1
:107F4000012B06D10121608800F0E0F801E01B2B35
:107F5000F8D037BD10B5054B0421187000F098F823
:107F6000FFF74CFDFEF770FB10BDC046B864FF1F65
:107F70000020F0B50BB20F0087B0834234DA274BF4
:107F8000187803F095FC051E2BD00378A02B25D183
:107F900003AE3100FEF7E4F8041E0BD1B378DB0723
:107FA00024D51F4B06341B68002B03D03100688892
:107FB00098470400A868002801D003F0A1FD002C18
:107FC00008D1184A039B1340174A934206D0B3784E
:107FD0001B2B03D00121688800F098F8280003F0DB
:107FE0005FFD80200002784007B0F0BD0F4B1B689A
:107FF000002B10D0310068889847041EDAD07378BF
:10800000002BD7D1B27801A90A704B800C71688817
:10801000FDF7F6FFCEE70624F1E7C046B864FF1F80
:10802000B064FF1F00FFFF0000011200B464FF1FD7
:10803000F7B50190FC200D0017001E0003F0E8FDCD
:1080400004001320002C12D0B02320002370089BC2
:10805000F4226770658026710830002B08D0190063
:1080600003F0B6FB2100019803F00AFE0020FEBDDC
:10807000089903F05DFCF5E710B5041E06D0007802
:10808000FD2803D803F08CFDFF23237010BD0000F2
:108090000A1F93B210B504000220032B05D88240BA
:1080A0000020024BD1529B189C7010BDD864FF1F5A
:1080B0000B8870B5043B04000D000220032B0BD885
:1080C0000121200000F04CFD03001420002B03D000
:1080D0002900200000F0DEFB70BD000007B5130092
:1080E000034A00920A00012100F02CFC0EBDC0469C
:1080F0001983001107B5019203220092024B0A0076
:10810000122100F049FC0EBD9783001107B56B46A4
:1081100001AA11800449D88008780633012802D1C9
:10812000190003F01DFC07BDB964FF1F0C4B10B50F
:1081300018700023FF210B4A1380138193819380D1
:10814000094A53801370517293819372D174D38210
:108150001375517703F0C4FD00F0FCF910BDC04663
:10816000E864FF1FD864FF1FBA64FF1FF0B58DB02D
:108170006B46002003910C229B5E834200DBB0E043
:108180005D4B187803F094FB051E00D1A4E0037842
:10819000902B00D09DE006AF01004688380000F02B
:1081A00013FA79680400002900D19CE03B88052B74
:1081B0006ED13B89032B1CD905AC200000F0A2F83E
:1081C0006288172A61D83989131D994231D179689B
:1081D000237804310291D90738D5607800F08EF900
:1081E000071E06D0002303712378012B08D0132B20
:1081F00023D0A868002800D178E003F081FC75E066
:108200006288029909A800F0A6F80290380000F0F0
:108210008BF909AA2378387A019200223100009262
:10822000029A00F012F9380000F064F9029B002B6A
:10823000DFD0300000F080F9DBE70378032BD8D1E2
:108240006288029909A800F0D6F8DEE7122B13D154
:10825000029909A800F0B5F8021EEAD127498B88D7
:10826000002BC6D0887909A9237801916178009103
:10827000310000F0EAF8BCE7002302AA9383300043
:10828000617809AAFFF72AFFB3E71D4B0993F6E7C8
:10829000042B02D09A1F012AABD8184A043B9B003A
:1082A000995A0029A5D0D218907831003A0000F0F0
:1082B000AEF800289DD13B88042B03D0012130006B
:1082C000FFF724FF012C04D1A868002801D003F097
:1082D00017FC280003F0E4FB8020039B00024340CE
:1082E00018000DB0F0BD012800D182E70121300057
:1082F000FFF70CFFEDE7C046E864FF1FD864FF1FDF
:10830000010017000B7803704B784370CB788A78A4
:108310001B021343438070470A88030002700A88D7
:10832000120A42700A88012A06D14A8882704A8855
:10833000120AC2700420704702208242FBD14A8890
:1083400004309A704A88120ADA708A881A718A8808
:10835000120A5A71EFE710B50400012082420CD9CD
:108360004B780A781B0213432380834206D1CB78D3
:108370008A781B0213436380002010BD022BFBD1BF
:10838000CB788A781B02134363804B790A791B02EE
:108390001343A380F0E70B8803700B881B0A43701C
:1083A0004B8883704B881B0AC3708B8803718B8842
:1083B0001B0A4371CB888371CB881B0AC3710820C9
:1083C000704703000120082A14D14A780878120265
:1083D00002431A80CA788878120202435A804A7986
:1083E0000879120202439A80CA79887912020243FC
:1083F0000020DA80704710B504000120022A05D160
:1084000000204B780A781B021343238010BDF8B577
:10841000060010200F00150003F0FAFB04000120F5
:10842000002C0ED0A0230C22290023806780201D61
:10843000002D07D003F0CCF92100300003F020FC20
:108440000020F8BD03F074FAF6E7F7B51E000090BF
:1084500008AB142017001D78019103F0D9FB041E0E
:1084600012D0A2230370019B47704380099B0571C2
:1084700046710C220830002B07D0190003F0A8F930
:108480002100009803F0FCFBF7BD099903F050FAB6
:10849000F6E737B5041E0FD04388002B0CD000251B
:1084A000C1881323007A172201950095FFF7CDFFAD
:1084B000FF2365806372257037BD000010B50C493D
:1084C00004004A88002A09D08B89002B05D000209F
:1084D000CB8A0222834201D010BD012213000A2060
:1084E000434300204032C854C81842800472F3E766
:1084F000BA64FF1F0023438003707047094B0021BB
:108500001A0010B55C88002C06D01C79844203D177
:108510000A234B43D01810BD01310A330329F1D18E
:108520000020F8E7BA64FF1F10B50400407A03F09A
:1085300037FBFF23637210BD7047043010B580B263
:1085400003F036FB002803D00421494203F028FA47
:1085500010BD000070B50025104CA0682580A581D5
:10856000A580A84202D003F0CBFAA56000250C4CF0
:108570000C4B606D1D80230058331D70A84202D043
:1085800003F0BEFA656500256068002801D003F09D
:10859000B7FA013508340A2DF6D170BD8065FF1F8A
:1085A0002465FF1F7465FF1F70B5041E09D1054DBA
:1085B0002880A881A880A868002802D003F0A0FA2B
:1085C000AC6070BD8065FF1FF0B54B8885B001932E
:1085D000002343600A7905000F00022A00D07BE0E7
:1085E000CA88032A17D98B685E7819783602DC7836
:1085F000D8790E4399781B7A24021B020C4303435B
:1086000053495BBA0B80331D93421ED1042C04D016
:10861000631F022B0ED9012015E0019A4D4B120168
:10862000D35A002B06D00198FFF7BEFF4A4A1369C0
:10863000013313610421B8682E812C80494203F074
:10864000AFF96860002005B0F0BD434D042C06D0A2
:10865000631F022B0FD9EB680133EB60DBE7019A54
:108660003C4B1201D35A002B05D00198FFF79CFF19
:108670002B6901332B61374B30000293019B029A27
:108680001B010193002301998C468B521300634414
:108690009C8003939E81FFF750FF039B041E98600C
:1086A00016D00421B868494203F07AF9FA8801002B
:1086B000043A200003F08CF80199029AFB888A5A48
:1086C000043B9B18029A8B522B6801332B60A2E764
:1086D000AB690133AB619EE71E4B0293019B1E0108
:1086E000029BF35A002B2DD002998C19A068002808
:1086F00028D0012A26D1FA889B189BB27352A189EF
:10870000994217D39B1AC018B96803F061F8029B0D
:10871000A289F35A934200D07DE700222B81A388DF
:108720002B80A3686B60029BF2520B4A53680133A3
:10873000536070E7084A9368013393600198FFF72C
:1087400033FF68E7044A536901335361F6E7C046D3
:10875000EA64FF1F8065FF1FF064FF1F70B5051EF0
:1087600015D10B4C0B4B1880230058331870606DDB
:10877000002802D003F0C4F9656525005035606813
:10878000002801D003F0BCF90834AC42F7D170BD29
:108790002465FF1F7465FF1FF0B51700A12285B087
:1087A000920001934243394B06001B680C009B1852
:1087B000D933FF331D78FDF741FF0430854204DDD6
:1087C0003000FDF73BFF0430C5B2BD4207D33A008D
:1087D00000213000019B03F043F805B0F0BD2900F3
:1087E000380003F01DF92300C6B250331E70039306
:1087F000019B29006365380003F042F9CBB2029374
:10880000002B02D0039B01361E700026230050333C
:1088100003931B78B34204D8606D002831D1002047
:10882000DBE7029A2800002A04D0013B1000B34283
:1088300000D02800F700E719387003F019F97860C4
:1088400000280ED03A78019902F0C2FF019A3B78D5
:108850000136D3180E4A0193D369F6B20133D361BE
:10886000D4E7039B18706065A74205D1084A13201E
:10887000D36A0133D362B0E7606803F041F908348A
:10888000F2E703F03DF900236365C8E73409FF1FF1
:10889000F064FF1FF7B50D0007000421686803F0BE
:1088A0007FF82B89040003702B891B0A43702B88E7
:1088B00083702B881B0AC3702E8902250436F6B2FA
:1088C000F42E15D81B4B9F4214D10C2003F0A0F9B5
:1088D0001135011E0CD0902303708E3B0371043BB5
:1088E0004380154B8460C680187803F0C9F90025D1
:1088F0002800FEBD5C237B43104AD31800935833F5
:1089000001931B78002B0FD103003200380000992F
:10891000FFF742FF019B05001B78002BE8D13800D0
:10892000009902F0EDFFE3E7054A0725536A01339A
:108930005362DDE7FEFF0000E864FF1F2465FF1FB0
:10894000F064FF1FF0B587B0009017200F001600ED
:108950000193FFF7F2FD1325041E19D00C98031E96
:1089600002D00199201D9847030AE370052302AA4B
:10897000A0700430908127700098667003A99380DE
:108980000494FFF787FF051E02D0200003F0B8F81B
:10899000280007B0F0BD0000F0B587B01F000CAB99
:1089A0001B780391059301210DAB06001C780492FE
:1089B00000F0D6F81425002821D02000FFF77EFD16
:1089C0000135041E1BD01149059B0A780370013242
:1089D000D2B2131EC68001D101231A000B7022717E
:1089E0003000049B03990097FFF7ACFF051E09D1E7
:1089F000230021000648074A093303F071F82800D4
:108A000007B0F0BD002363802370F8E7EC64FF1F1C
:108A10009384001130750000F8B505000E00064C77
:108A2000064F2368002B02D03100280098470434F9
:108A3000BC42F6D1F8BDC0469065FF1FA465FF1F7C
:108A40000123064A5B425380002313715362044A98
:108A5000136053609360D36013617047A465FF1F78
:108A60009065FF1F0200002310B506499C000859BD
:108A7000002801D1625010BD0133052BF6D113201F
:108A8000F9E7C0469065FF1F034A5388181A43420E
:108A90005841404210407047A465FF1FF0B585B0B3
:108AA00002930AAB1F780CAB1B88009008000E00E5
:108AB00001920393FFF7E8FF05001120002D1BD161
:108AC0000E48FFF7E1FF04001520002C14D0062209
:108AD0000B99A771E01D02F07BFE019B3000237112
:108AE000029B29006371009B66802370039B656273
:108AF000E381FFF791FF280005B0F0BDFFFF000004
:108B000010B5FFF7C1FF04000220002C12D06088CE
:108B10000121FFF781FF606A002801D002F000FF09
:108B200028220021200002F003FF012300205B42E5
:108B30006380207110BD000030B5074A074C55888E
:108B4000010013780020A54204D05B1A59424B4122
:108B50005842104030BDC046A465FF1FFFFF000013
:108B6000084A10B501230C00904208D0FFF78CFF93
:108B7000031E04D0037923405A1E9341DBB2180030
:108B800010BDC046FEFF0000024B1879431E9841FD
:108B9000C0B27047A465FF1F70B504000D00160039
:108BA000FFF772FF002804D10D4B9C4200D0143017
:108BB00070BD416A03790520002907D012221A40AE
:108BC000102A02D10520002EF2D10F20DB06EFD5AE
:108BD000897E0C20A9428941494249420840E7E781
:108BE000FEFF0000030010B5002800D110BD0348AF
:108BF000034A41889142F9D09847F7E7A465FF1FDF
:108C0000FFFF0000002330B5C45CCD5C6C40D45441
:108C10000133102BF8D130BD0F23002210B5C45CF6
:108C200064002243CA54C25CD209013BF7D210BD92
:108C30000200010010B52032103102F0F1FD10BD2C
:108C4000F0B58BB00390102005931700049102F04B
:108C5000A7FD0090102002F0A3FD009B13240190BB
:108C6000002B05D000280CD11324009802F058FEE8
:108C7000019B002B02D0180002F052FE20000BB026
:108C8000F0BD102002F08CFD0600102002F088FDDF
:108C900013240500002E00D1AEE0002819D01022C8
:108CA000002102F045FE32002900039802F0B8FDD1
:108CB000041E0ED133787F2B51D830000099FFF776
:108CC000ABFF009B1B787F2B53D801990098FFF7CF
:108CD000A3FF300002F024FE002D02D0280002F095
:108CE0001FFE002CC1D1102002F05AFD06001020FA
:108CF00002F056FD0290002E7CD0002878D03A0079
:108D00000F3223000125121105D00F333B4015B25D
:108D10005A4253411BB26A1E1201002B33D0049BEE
:108D2000D2B298180099029AFFF76CFF013D102209
:108D30000021300002F0FCFDADB2049F2D017D1931
:108D4000AF4242D0002C33D0300002F0E9FD029B4C
:108D5000002B00D189E7180002F0E2FD85E7290029
:108D60003000FFF759FF28002549009AFFF74AFF16
:108D7000A7E729000098FFF74FFF28002049019A34
:108D8000FFF740FFA5E70F210F4004998A18D9B2D9
:108D90008F4208D9D15C06A819540133102BF6D1A3
:108DA000029A0199C0E7791A48424141C901F2E7A4
:108DB0003900300006AAFFF725FF3200039806A904
:108DC00002F02EFD10370400BAE7002CBCD13000B1
:108DD000029906AAFFF716FF320006A9039802F0CF
:108DE0001FFD082204003100059802F0F1FCABE7FA
:108DF0001324A9E71324AAE7002800D06EE733E77D
:108E000098BF0011F0B58BB00F001600022500903E
:108E100000283FD0002A3DD00B1DDBB21800029382
:108E200002F0BEFC1135041E34D0FDF747FD0500ED
:108E30003A000099201D02F073FEEBB20393E37039
:108E40002B0CDBB22F0A00936370FFB22B0E237042
:108E5000A7700193FDF72CFD1022010006A802F077
:108E60005FFE2100029A04AB06A8FFF7E9FE051E8B
:108E70000DD1039B08223370009B04A9B370019BA2
:108E80007770F370301D02F04BFEFDF71DFD2000E2
:108E900002F046FD28000BB0F0BDF0B58FB00D001C
:108EA000149E039004920593002A03D1022420000B
:108EB0000FB0F0BD002EF9D00398FFF7E5FD1424A4
:108EC000071EF4D07278337812021A43B3781B0469
:108ED0001343F27812061A43036A0192934201D3B4
:108EE0000133E3D1002D03D03B7901249B07DED56C
:108EF0000822002106A802F01BFD059B1324043361
:108F0000DBB21800029302F04BFC051ECFD0059A8D
:108F10000499043002F004FE04223100280002F01B
:108F2000FFFD3900102210310AA802F0F9FD2900D6
:108F3000029A06AB0AA8FFF783FE041E0FD108228F
:108F400006A908A802F0ECFD0822311D08A802F0CD
:108F5000DFFE012807D101990398FDF7C9FC28001D
:108F600002F0DEFCA3E70124F9E7000070B51C4C19
:108F700005002368181E10D0002D14D11A78002A7D
:108F80000CD1981C083202F023FC02F0C9FE013516
:108F9000002808D123681D70012070BD0A33180015
:108FA000082202F015FC2368002BF5D0122002F0F5
:108FB0002FFE061E0DD0C1232168037045700231BB
:108FC0001022023002F004FC23683100587802F0CD
:108FD00057FE206802F0A4FC00232360DCE7C046B3
:108FE000CC65FF1FF8B504002020FDF755FB0D4EA2
:108FF000A700BB590500002B0DD000280BD0D87856
:10900000FF2809D108492A000C55F35907480333B2
:10901000611802F065FDF8BD290002F059FC002836
:10902000F0D1F8E7E865FF1FD065FF1F3DA20011F2
:1090300070B5064D84006359002B05D0D87802F036
:10904000AFFDFF226359DA7070BDC046E865FF1FAF
:1090500070B506008CB00C00150000213022684667
:1090600002F066FC31001022684602F059FD1D2016
:1090700021000322684402F053FD6846FFF7D8FD43
:109080002D21040003222800694402F049FD20003C
:109090000CB070BDF0B50700160097B001931CAB83
:1090A0001D7830221EAB00910AA800211C7802F026
:1090B0003FFC102239000AA802F032FD10220021E4
:1090C00002A802F035FC0722310002A802F028FDB8
:1090D000072202AB9818631E9C41019902F020FD03
:1090E00002AB9C732B005A1E934102AAD37300213A
:1090F000102206A802F01CFC06221D9907A802F007
:109100000FFD1A2002ABC01806221F9902F008FDBD
:10911000102200990EA802F003FD102202AB0EA946
:1091200008781C78013A6040D2B2087001330131EE
:10913000002AF5D10AA8FFF77BFD102212A904002E
:109140000EA802F045FB102206AB0EA908781D7888
:10915000013A6840D2B2087001330131002AF5D1DA
:109160000AA8FFF765FD044310222098E4B212A973
:1091700002F0D6FC200017B0F0BD70B50E00140050
:109180008CB00100102268461D0002F0C9FC3100BD
:10919000082204A802F0C4FC2100082206A802F05C
:1091A000BFFC6846FFF744FD04001022280008A910
:1091B00002F0B6FC20000CB070BDF8B506000D0042
:1091C00000243719AC4200D3F8BD02F089FB030A32
:1091D0003B70631CDBB201379D4203D90234F0546B
:1091E000E4B2EEE71C00EDE773B506000C000225C3
:1091F000002819D0002917D0032101A8FFF7DDFFAF
:109200006B469A793F231A40013313436A46300074
:10921000937101A92200FFF71BFF051E04D1032251
:10922000E01C01A902F0D4FA280076BD03785807A3
:10923000DA08C00FD20080009B0710439B0F184331
:10924000C0B2704707230B40C908C9000B43037025
:109250007047000070B50400FFF7EAFE134DA4004C
:109260006359002B21D0186A002801D002F058FB66
:109270002B59986E002801D002F052FB2B59D86E62
:10928000002801D002F04CFB2B59186F002801D0A8
:1092900002F046FB2B59586F002801D002F040FB2A
:1092A000285902F03DFB00232B5170BDE865FF1FDC
:1092B0000E4B8000C35870B50C00002B0FD09D687A
:1092C000002D0CD02B78201D0B706B784B70A97C77
:1092D000FFF7B8FF2B7E23726B69E36070BD10222D
:1092E0000021200002F024FBF8E7C046E865FF1FDC
:1092F000014B18607047C046E465FF1F074A030032
:109300008000825810B5002A06D0D088984203D138
:10931000012901D1FFF79EFF10BDC046E865FF1F80
:10932000F0B5264E95B087000B93BB590500099107
:1093300012200A92002B31D0D888FFF7A5FB040039
:109340001420002C2AD0280010A9FFF7B1FFBB5928
:109350001E781D6A002E23D00895FDF7EFFA07004E
:109360000020FDF7F1FA0790A379E61D069310ADF2
:109370000CA9089800F0E2FA0EA9280000F0D7FA2C
:109380000B9B0A990493069B09980293079B0396EB
:10939000019300970EAB0CAAFFF77CFE15B0F0BD51
:1093A000FDF7CCFA06903000FDF7CEFAE31DA77961
:1093B000079310AB06000893DAE7C046E865FF1F85
:1093C00030B50C4C85002A59030085B00120002AD5
:1093D0000ED018006946FFF76BFF2B591A78D88812
:1093E000054B002A00D1054B6A46072100F0D9FB46
:1093F00005B030BDE865FF1F2F9900113D990011A0
:1094000030B5094C8500295985B0102268462531B0
:1094100002F0DEF92A591121044BD0886A4600F087
:10942000C0FB05B030BDC046E865FF1FD9990011EB
:1094300030B5094C8500295985B010226846353170
:1094400002F0C6F92A591121044BD0886A4600F06F
:10945000A8FB05B030BDC046E865FF1F179A001194
:10946000F7B54D4F86001020F4590D0002F098F921
:10947000F3592062186A132200286CD0033A29009D
:109480009C6802F0A5F9F3591A780192002A58D184
:109490001E6A227D317B944651400122019F114278
:1094A00001D167461740217D914339432175377BB0
:1094B0004F40BC4660460027800701D44F08174044
:1094C000012102208F40227D82433A432275377B5F
:1094D0005740BC4660460027400701D497080F401C
:1094E0000420227DBF0082433A432275627D00271B
:1094F00094466046727B42400A4201D167460F4063
:109500000121627D8A433A436275777B5740BC46AE
:1095100060460027800701D457080F400220627D73
:109520007F00824317436775767B00227E40760773
:1095300001D4BA080A400426617D9200B1430A436F
:1095400062756A78002A08D06278002A05D0052260
:109550000533DA7700221000FEBD0422297911427A
:1095600005D1A17C114202D10533033AF1E7019AFA
:1095700021782C78002A02D10A0021001400182238
:109580000429E8D8042CE6D805206043034A0533B3
:109590001218525CDDE7C046E865FF1FA8BF001146
:1095A00010B50A001121024B00F0FBFA10BDC046B5
:1095B000739A00110B0030B587B001AD2B806B465C
:1095C00004001100981D082202F002F92A000B2164
:1095D0002000024B00F0E5FA07B030BD9B9A001165
:1095E00010B50A001121024B00F0DBFA10BDC04695
:1095F000EF9A001113B50B0011006A4613706B4609
:1096000004000622581C02F0E3F86A4608212000F4
:10961000014B00F0C6FA13BD0F9B001110B50A00F4
:109620001121024B00F0BDFA10BDC0465F9B001136
:109630007FB505000B4BAA00D4580800002C0FD0B2
:10964000666F237FE28821780396266F0296E66E86
:109650000196A46E0094FDF709FC2800FFF7FAFDBF
:109660007FBDC046E865FF1F10B51721FFF7E0FF7B
:1096700010BD000070B50A000D00064B0221040069
:1096800000F08FFA060029782000FFF7D1FF3000A4
:1096900070BDC0463F9A001170B586B000236A467F
:1096A0001370836804001D78681E0A2859D801A920
:1096B00002F086F8060633373B3F43474B4F5300D3
:1096C000180000F042F9062312284BD000281BD1C5
:1096D0006088FFF7D9F90823002813D04279002ABF
:1096E00047D1264B1A78072312070BD5244B1A684B
:1096F0000723002A06D01668002E03D0290001AAED
:10970000B04703006A4613706B461B786088002BD5
:109710002AD1FFF767FC06B070BD180000F06CF9A5
:10972000D4E7180000F087F9D0E7180000F093F9AB
:10973000CCE7180000F0ADF9C8E7180000F0C3F955
:10974000C4E7180000F0F6F9C0E7180000F0F6F9D9
:10975000BCE7180000F013FAB8E7180000F013FA9D
:10976000B4E707236A46137069466088FFF782FFF3
:10977000D1E70523012AC5D1024BB8E77564FF1F65
:10978000E065FF1FE465FF1FF8B52C4F8600F35915
:1097900004000D00002B40D0DA8882423DD15A7877
:1097A000062A33D11A78002A2ED0012099681A6A25
:1097B000097D014206D0157B054203D007225A706D
:1097C0000120F8BD0220014204D0157B054201D0E2
:1097D0000922F4E70420014204D0127B024201D0A6
:1097E0000B22ECE7164B1B68002BE9D05B68002BC3
:1097F000E6D020009847BB5900215B78122BDFD1BF
:109800002000FFF715FFDBE70E4BECE7112A04D130
:10981000002900D032252900F2E7002D08D12000D0
:10982000FFF732F9002803D01023027913430371A4
:1098300021002800FDF798FAC2E7C046E865FF1F3F
:10984000E065FF1FE465FF1F70B50E4E8500AB5944
:109850000400002B13D01B78002B11D10A4B1B687E
:10986000002B04D05B68002B01D02000984773596F
:109870005B78122B03D100212000FFF7D9FE70BDC9
:10988000024BECE7E865FF1FE465FF1FE065FF1F83
:10989000094B8000C3581020002B0CD01A6A002AF4
:1098A00009D09B68002B06D0127A1B7E101C9A42AE
:1098B00000D9181CC0B27047E865FF1F70B50300DF
:1098C0000D0014000220002A30D000292ED0137081
:1098D0000B78081D53704B789370FFF7A7FCE0706E
:1098E000012002212B7A23716B7B034063716A7B19
:1098F0000A401343042263716E7B16403343637145
:109900006E7BF608F600334363712B7B0340A37133
:10991000287B014000200B43A371297B0A4013439D
:10992000A3712A7BD208D2001343A37170BD10B576
:109930000A0001000120FFF7C1FF10BD10B50A00A9
:1099400001000220FFF7BAFF10BD70B506000C0041
:109950000220002E30D000292ED07378201D0B70ED
:10996000B3784B70F178FFF76DFC012235792572E1
:1099700071794B1008001340934010400343881046
:1099800010408000C9080343C9000B436373B179D9
:109990004B100800134093401040034388100240CE
:1099A0009200C9081343C9000B4321202373FCF71D
:1099B00073FE854201D2122070BD2220257AFCF769
:1099C0006BFE8542F7D823781820042BF4D86378EF
:1099D000012BF1D80020EFE7030010B50220002989
:1099E00009D0002B07D00322481C0A7019000D3241
:1099F00001F0EEFE002010BD03000222080010B5A9
:109A0000002B06D0002904D00E32591C01F0E0FED4
:109A10000022100010BD030010B50220002909D05B
:109A2000002B07D00422481C0A7019000C3201F0E8
:109A3000CFFE002010BD10B5FFF7DEFF10BD030004
:109A40000220002906D0002B04D0052200200A7035
:109A50001B784B70704703000220002B08D00029B0
:109A600006D05B7800200B70013B082B00D9183022
:109A70007047030010B50220002909D0002B07D041
:109A80000622481C0A7019000A3201F0A1FE0020CB
:109A900010BD10B5FFF7B0FF10BD02000B00022093
:109AA00010B500290ED0002A0CD00721197011889A
:109AB00059701188090A997011180822D81C01F0F0
:109AC00087FE002010BD03000A00022010B5002B05
:109AD0000CD000290AD099785878090201431180E6
:109AE000901CD91C082201F073FE002010BD030059
:109AF00010B50220002909D0002B07D00822481CED
:109B00000A701900921801F063FE002010BD0200D7
:109B10000B00022010B500290BD0002A09D0092122
:109B20001970117818185970511C062201F050FE56
:109B3000002010BD10B5FFF75FFF10BD02000B0045
:109B4000022010B5002A09D0002907D051781970D9
:109B500011180622581C01F03BFE002010BD030026
:109B600010B50220002909D0002B07D00A22481C7A
:109B70000A701900063201F02BFE002010BD10B54E
:109B8000FFF73AFF10BD02000B00022010B5002ABB
:109B900006D0002904D018005178FFF753FB0020AD
:109BA00010BDF0B585B017001E006A4606230500FB
:109BB000080091819380FEF7C0FC1324011E0290DF
:109BC0000CD03800B047041E05D1280001A9FEF7CB
:109BD0006FFA041E02D0029801F092FF2800FFF7EE
:109BE00001FA200005B0F0BDF0B504008BB0019182
:109BF00015000021102202A801F09AFE334EA700A2
:109C0000B85900283CD0C388A34239D10378002B2F
:109C100036D14278062A18D102000100553235317A
:109C20000C3006ABFFF7A9FA002829D12000FFF776
:109C30002FFE020006A902A801F0CAFD200002A919
:109C400001F066FD01200BB0F0BD816E002917D038
:109C50000B8A112A28D19D420ED101981231093A5E
:109C600002F056F8012807D1BB5920009D6EFFF77E
:109C70000FFE29000200DEE732212000FFF7D8FCAA
:109C80002000FEF701FF061E1BD0416A002918D0F4
:109C90000B8AAB4215D108220198123102F038F834
:109CA00001280ED1716A0AE09D42E9D1082201988B
:109CB000123102F02DF80128E2D1BB59996E8A7E4B
:109CC000B9E7200001F064FDBCE7C046E865FF1F6E
:109CD000F0B56B4D87007E5985B0337802900393C1
:109CE000002B00D087E0B368346A019370780628AF
:109CF00017D101221B7D134202D0217B114218D1C2
:109D00000222134202D0217B114251D1042213427C
:109D100003D0237B134200D08BE0019B5A7DEB598B
:109D200091E007380428F8D801F04AFD032E426775
:109D30008300B36E002B03D11C2001F031FDB0660F
:109D4000EB599C6E002C1CD010220021200001F049
:109D5000EFFD0298FFF79CFD01002000FFF72DFAB0
:109D600001F0BEFD2082200008211230FFF725FA05
:109D70000298FFF78DFDA076EB592100D888FFF7F8
:109D80000FFC0822EB591CE0B36E002B05D01A0023
:109D9000198AF0881232FFF70DFC0222019B197D0F
:109DA000EB5911423DD0207B10423AD0073208E0F7
:109DB000F488FCF7DBFD01002000FFF711FC0A220C
:109DC000EB595A70029B9C002A595378073B042B8D
:109DD00011D8D088FEF758FE00284ED0C3895A0803
:109DE000D2182849029B0298CB542B5941180433AE
:109DF000254801F075FE05B0F0BDFCF79FFD03009E
:109E00000120834201D100200393EB59DE88FCF747
:109E10009BFD039902003000FFF7ECFB019AEB5920
:109E2000117D042211420CD0217B114209D00B225A
:109E3000C7E7F688FCF73CFD01003000FFF7EEFBBA
:109E40006BE7019A527D01210A4204D0607B0842EF
:109E500001D00C22B5E702210A4204D0607B0842FF
:109E600001D00E22ADE704210A4204D0627B0A42EF
:109E700001D01022A5E71222A3E7FA225200B0E790
:109E8000E865FF1FEC65FF1F47A2001110B5064BE8
:109E90001A780423100018401A4200D00348FFF734
:109EA00027FA002010BDC0467564FF1F2043FF1F26
:109EB00070B50400FFF7D4FA051E43D12000FFF768
:109EC0007FFA234EA400A0598268937CDB0708D553
:109ED0000321036A1B790B40012B02D1017F0B4345
:109EE0000377431DD97F8B1E022B0DD8022900D08A
:109EF0000121C088FCF790FF042133591A7F597063
:109F00000A431A77280070BD01290CD102231022C0
:109F1000437000210C3001F00BFD30591021353019
:109F2000FFF74BF9EEE70529ECD10223D118437076
:109F300010220C3001F04CFC04233259117F0B43EA
:109F40001377EAE708251828DCD1053DDAE7C04693
:109F5000E865FF1FF0B58BB0059143887E4F9E00EA
:109F6000F45915000493002C15D1012902D00020CA
:109F70000BB0F0BD101D57781678FFF757F9EB6856
:109F8000320002932B7A0499019300903B00200049
:109F9000FCF70CFFEBE7E388049A934201D008201A
:109FA000E6E72378012B00D1D4E0059B581E092851
:109FB00000D9CFE001F004FC05CE0A29CC506C8515
:109FC0009AB229000498FFF773FFD1E72000290017
:109FD0001022453001F0FCFBB9594B78042B02D11B
:109FE000013B4B70C3E70B000A00253335320C31BF
:109FF0000498FFF795F90498FFF702FA0522431E2B
:10A000009841BB59C0005A70B2E7200029001022C5
:10A01000553001F0DDFB049B4F4C9D0029590498FD
:10A020000A0006AB55320C31FFF77AF92959102294
:10A03000453106A801F06CFE012808D10498FFF70D
:10A04000F7F90590002804D106222B595A7005987B
:10A050008EE708230593FAE763780C2B7AD1E36E39
:10A06000002B03D11C2001F09BFBE066BB59D86E8E
:10A0700000286FD01022290001F0AAFBBB590498D8
:10A08000DC6EFFF705FC0D22A076BB595A706EE717
:10A09000E06E00285ED063780D2B5BD12B88082200
:10A0A0000382A91C123001F093FBBB599A68517DC1
:10A0B0000222114226D0186A407B104222D00C3274
:10A0C000E4E763780E2B45D1236F002B03D11620D4
:10A0D00001F066FB2067BB59186F002803D01022DF
:10A0E000290001F075FB0F22BB59CFE763780F2BD6
:10A0F00030D1206F0622691C103001F069FBBB597A
:10A100009A68517D0422114203D0196A497B114299
:10A11000D5D100210498FFF78BFA28E7636F002B55
:10A120000DD0BB59586F0028F3D01022290001F040
:10A130004FFB0122BB5952425B6F1A61E9E71420C1
:10A1400001F02EFBBB5960675B6F002BE9D126E75E
:10A150002978DFE707200BE7E865FF1F10B5064CFD
:10A16000207001F015FC06212078FDF791FF0348CF
:10A17000FEF778FC10BDC046FB65FF1FFD92001185
:10A1800000200BB270B50D00834216DA264B18780A
:10A1900001F08EFB041E0DD00378922B0ED0A02B65
:10A1A00037D0224B1878FF283AD0210001F068FD03
:10A1B000002835D180200002684070BD43780E2B06
:10A1C0000BD03E2BEDD18378052B12D0082BE8D194
:10A1D00081798088FFF7D8FA08E0154B82889A4287
:10A1E000DFD183681878591CFEF7C0FE002817D10C
:10A1F000D7E7104B1B785B0712D50F4B1B68002B62
:10A200000ED09B68002B0BD0C289811D8088984797
:10A21000ECE7FFF741FAA068002801D001F070FCDC
:10A22000200001F03DFCC5E7FB65FF1F1943FF1F40
:10A23000182000007564FF1FE465FF1F10B500784B
:10A24000FFF712FA10BD10B50078FFF7FDFA10BD48
:10A250000C234343084A10B59B185A68002A03D0C0
:10A26000012901D1904710BD9B68002BFBD000292C
:10A27000F9D19847F7E7C0461866FF1F01238340CE
:10A28000094A10B5946B1C439463506B9843506318
:10A29000D46B20009843012901D120001843D063DA
:10A2A000116B0B43136310BD00800040F0B5002418
:10A2B0000127154B85B0DA6B144E03921A6C01928C
:10A2C000DA64019BE3403B4217D0039DE5403D40EB
:10A2D0000295E5B202992800FFF7BAFF316A736A66
:10A2E000002908D03900002B01D0029979402800BC
:10A2F000FFF7C4FF01E0002BF9D101340C36172C15
:10A30000DFD105B0F0BDC04600800040FC65FF1FF6
:10A31000064B01215A68C2400A4204D01B68C34060
:10A320001800084070471B6DF9E7C04600800040E8
:10A330000122064B8240002903D0D9680A43DA6023
:10A340007047D9689143D960FAE7C04600380040A9
:10A3500030B5032444430F4BE25C1B199C785D78B5
:10A3600001232D1B0135AB40013BA340A140DB4342
:10A370000C00122807D80849920052181168194099
:10A380002143116030BD054A11680B40234313601F
:10A39000F8E7C046EFBF001108F0004014F000409D
:10A3A000C21F70B5D4B20623092C0BD80125084C66
:10A3B0009540002908D00021FFF7CAFF23682B43EE
:10A3C00023600023180070BD2368AB43F8E7C04644
:10A3D00000380040214BF0B51B185B78022B21D1CF
:10A3E000032444431E4A1F4EA35C12199478012291
:10A3F00015008540B76B013CE4B23D43A240B56314
:10A40000194C122815D89B0000290CD117495B184C
:10A4100099680A439A600123205C154A83401168B9
:10A420000B431360F0BD11495B1899689143996023
:10A43000F1E70E4B00290DD159690A435A61225C9C
:10A440001328E8D00123203A93400A4908680343BF
:10A450000B60E7E7596991435961F0E7FC65FF1F1D
:10A46000EFBF00110080004034C0001100F0004038
:10A47000A0F00040A4F00040F8B500241B4E1C4D95
:10A480001C4B1B5D012B1FD1194A9269E2401A42F5
:10A490000BD00122B25693402200143AD2B2022AC3
:10A4A00009D815494A6913434B61013402360C350A
:10A4B000172CE5D1F8BD0022B2560F499200521870
:10A4C00091680B439360F0E7022BEED1E7B23800BE
:10A4D000FFF71EFF01235840C1B23800FFF77AFF93
:10A4E0003800FFF715FF6877DFE7C046C1BF0011EE
:10A4F000FC65FF1FFD65FF1F00F0004001220238D0
:10A500008240054B002903D059690A435A617047BC
:10A51000596991435961FAE700380040F8B50E00D7
:10A5200001210F008740114A0400D368FD43BB435B
:10A53000D360831E8B4201D8FFF7E0FF002120008B
:10A54000FFF72EFF0A4A0B4B5168012E05D1394304
:10A550001B1951605E700020F8BD29405160022235
:10A560001C1962709A6915409D61F4E7003800403B
:10A5700000800040FC65FF1F012210B58240074BA0
:10A58000002906D019680A431A600121FFF7C6FFA7
:10A5900010BD196891431960F7E7C046008000407C
:10A5A0000C2370B5002543430A4A29009B181D70EF
:10A5B000094B04001B185D70FFF7B0FF0123A34097
:10A5C000064928000A681A430A6005490A689A433E
:10A5D0000A6070BD1866FF1FFC65FF1F34800040D5
:10A5E0003080004070B504000E00FF2813D0032512
:10A5F0000540FFF7D5FF084AA3089B009B183F22A0
:10A60000ED00AA40AE401968200091433143196023
:10A610000121FFF78DFE70BD18380040F8B50C24FD
:10A620004443134B0500E4186368002B03D1A3686F
:10A630001220002B1AD0022201270E4B00215B1999
:10A640005A7028002770FFF769FF63681E1E08D044
:10A65000A3683E00002B04D02800FFF759FE4640B7
:10A66000F6B228003100FFF709FE0020F8BDC04611
:10A670001866FF1FFC65FF1FF7B5C420FF222B4B98
:10A6800080001958002491433F3A0A431A5080220F
:10A69000274F5202274E1A60274B1D5D002D21D0F7
:10A6A000A31E012B03D80121E0B2FFF727FF012DE4
:10A6B00018D11F4B9B69E3402B4213D0E3B2180023
:10A6C0000193FFF725FE01000198FFF755FFE3B264
:10A6D000143B022B1DD801217156184A8D40536935
:10A6E000AB4353613B7F002B0DD0E5B22800FFF751
:10A6F00095FF2800FFF70CFE7B7F0100834202D00C
:10A700002800FFF7A5FD01340C370236172CC3D102
:10A71000F7BD012100237156F3568D40074A9B0077
:10A720009B189A68AA439A60DCE7C04600E100E003
:10A73000FC65FF1FC1BF0011FD65FF1F00F0004059
:10A7400070B50E0015000400FFF72AFF0C236343C9
:10A75000094A20009B189D605E60FFF75FFFF021B3
:10A76000064B074A8900051E5A5002D02000FFF709
:10A7700017FF280070BDC0461866FF1F0000FF1FAE
:10A78000ADA2001170B5134D07202C78002C1FD1FD
:10A79000982221005200280001F09AFA0123C420D7
:10A7A000FF222B700C4B80001C635C630B4B1C6006
:10A7B0005C600B4B195891433F3A0A431A50802270
:10A7C00052021A600D20074A074901F011F82000D3
:10A7D00070BDC046FC65FF1F00800040A0F0004037
:10A7E00000E100E079A6001179A40011030010B582
:10A7F0000620072B09D8054A137001F041F8D7212C
:10A800000020034B034A89005A5010BD4843FF1FE4
:10A810000000FF1F911BFF1F70B51D0002240C29B3
:10A8200010D8094ACA40D2070CD5FBF741FF041ED5
:10A8300008D1059A04992800FBF756FFFCF7C4FDE0
:10A84000FFF724FB200070BD1210000030B50D781A
:10A8500002232C009C43184201D02B431C000825E6
:10A860002300AB43284201D02B00234320241D00AA
:10A87000A543204201D01C4325002A230D70184215
:10A8800004D011781E3B0B43137030BD0028FCD15F
:10A890000C2113788B43F7E7F8B51D0006AB1B8836
:10A8A000140007AA0E000B201778002B27D10A7876
:10A8B000022A49D14A68507811780002244A084394
:10A8C0008018042840D800F07BFF03121D1B2300D2
:10A8D000F06801F045F9021CC0B2B84200D93A1C38
:10A8E000D2B22000F1682A8000F072FF06E0022256
:10A8F000F3681B882A8023701B0A63700020F8BD50
:10A900000622EEE701232B80F3681B782370F5E71E
:10A91000F368002B16D008222A801A8822701A8821
:10A92000120A62705A88A2705A88120AE2709A88D3
:10A9300022719A88120A6271DA88A271DB881B0A76
:10A94000E371DBE72B80D9E701202B80D7E7C046F6
:10A9500000D6FFFFF7B516000A781D0008AB1F8868
:10A960000C000123022A18D14A685078117800029D
:10A970002B4A0843801803280FD800F021FF022536
:10A980004439E06801F0ECF8C0B20723B84204D3C0
:10A990007B190193152B02DD0D231800FEBDE06825
:10A9A0002A003100C01900F013FF6B4600209B887D
:10A9B000E268D0541B4B1B68834203D01B68834260
:10A9C00000D098470023E8E70B23002FE5D1022DA4
:10A9D000E2D1737832781B021343E2681380114B83
:10A9E0001B68002BEED01B68002BEBD00120E8E7A2
:10A9F0000B23002FD1D1062DCED12A003100E068E3
:10AA000000F0E6FEDEE70B23002FC6D1012DC3D1F7
:10AA100032787533012AC0D8E3681A70D2E7C0468D
:10AA200000D6FFFF0868FF1F70B50C00150007284F
:10AA300037D800F0C5FE041436361B36242E1820F5
:10AA400015290BD8184E16220021300000F070FF97
:10AA500022002900300000F0BBFE002070BD18204D
:10AA60000229FBD11288114B1A80F6E71820082919
:10AA7000F4D10A000E48290000F0C2FFEDE71820CB
:10AA80000129EBD10B4B10780B49DA69FFF7DEFE99
:10AA9000E3E718200129E1D1064B10780749DA6B6A
:10AAA000F4E70220DAE7C046F067FF1FC643FF1F46
:10AAB000BC43FF1F4C43FF1F7443FF1F9443FF1F02
:10AAC000030010B50020DB0704D50721024A034824
:10AAD00000F08CF810BDC0464CC000114C43FF1F65
:10AAE000054A03001068002803D082889A4201D1E9
:10AAF000806870470068F6E7006AFF1F0A88030055
:10AB000008009A4204D08A8804309A4200D000207B
:10AB100070470000F8B5F22200230D4F0D4E796802
:10AB2000050042433370994200D07B600A4C0021FB
:10AB3000200000F0FDFE00231A007C60AB4202D131
:10AB400000203370F8BD01332280DBB2F234F5E728
:10AB5000F86AFF1FF66AFF1F046AFF1F73B56B4692
:10AB600001900600684615001980FCF75FFF041E7F
:10AB700011D1002D0FD07689002E11D00C2000F0BD
:10AB80000FFE00280ED0084A046013688680856096
:10AB9000002B02D11060200076BD1A001B68F7E779
:10ABA0000224F8E71324F6E7006AFF1F01210022C0
:10ABB0000A4B10B549420A4C198099809A719A70D3
:10ABC000084B2070012019805A60FFF7A3FF2078FE
:10ABD000FCF78AFF0448FDF745FF10BD1068FF1F12
:10ABE000006BFF1FF86AFF1F99AC0011022310B51C
:10ABF000002802D0FFF7B2FF0300180010BD0000CC
:10AC0000030010B50020DB0704D50421024A0348E5
:10AC1000FFF7A4FF10BDC04660C00011CC43FF1F6A
:10AC2000F0B50E2687B003930CAB1F8802ABF61865
:10AC30000500080031000292FDF77AF804000120B7
:10AC4000002C0FD03088FFF74BFF03000E20002BA5
:10AC500008D05E68002E05D021002800039B029AD0
:10AC60000097B04707B0F0BD0A4B10B5984207D126
:10AC70000122002352420A808B708A808B7110BDA2
:10AC8000FFF73CFF0028FAD001235B42038000233A
:10AC90008370F4E7FFFF0000F8B5050001290AD131
:10ACA000134E00243388F227AB4219D028001149F3
:10ACB000FFF7DAFF06E0022904D10139FDF750FF62
:10ACC0000028EDD0F8BD3B0063437268D018D35A1A
:10ACD000002B09D03A00002100F02AFE0134E4B232
:10ACE000054B1B78A342EED801235B423380DDE79E
:10ACF000F86AFF1F1068FF1FF66AFF1F10B5FFF705
:10AD0000FDFE03000020834200D0987810BD0000B3
:10AD1000F0B589B01C000EAB80CB03901E8810AB41
:10AD20001B78049202930B7A0D00DB0616D42B7865
:10AD30000593022B24D00498FFF7D2FE002812D0EE
:10AD400003689C46002B0ED0029B22000193290031
:10AD50003B00644603980096A04705E00498FFF77F
:10AD6000BFFE002802D10E2009B0F0BD8368002B81
:10AD7000F9D00A222900039898470028D7D0F3E792
:10AD80006B6858781A786B4B000210439842D2D8FF
:10AD9000043B984210D2684B984242D015D8674B7A
:10ADA000C0180128C7D80B20002EDDD1EB681A7817
:10ADB00059683A80200028E0614BC018032800D968
:10ADC00079E000F0FDFC846A789E5E4B9842B2D137
:10ADD0000B20002EC8D101233B80EB6831001B788B
:10ADE00023706889013080B2FCF7A2FF3A88031E05
:10ADF0000ED0017802328A183A8042896270428904
:10AE0000120AA27059680278E01C00F0E1FC06E02A
:10AE100004323A8031000422601C00F089FD0020D9
:10AE2000A2E70B20002E9FD1EB6807A91E88042300
:10AE30003B80330A300026706370FCF779FF051EF3
:10AE400028D004AB9A890E2304A95B183E49C66832
:10AE5000FCF7E2FF00280BD12B783C486A68059983
:10AE6000FBF798FB002803D1012304AA5B42D3819E
:10AE70003278022A06D17168201D00F0A9FC3B88B7
:10AE800002333B800E2304AA9B181B88A3701B0A65
:10AE9000E370C4E704ABDE81F4E70B20002E00D0A2
:10AEA00062E7E9680398FFF729FF02233B802070DF
:10AEB000000A6070B3E70B20002E00D054E7022296
:10AEC000EB681B883A8023701B0A6370A7E7E86869
:10AED00000F046FEC2B203000720B24200D243E7B0
:10AEE0000DD00299DBB27118994202DB921BD3B2EA
:10AEF0000293029BE9681A003B8089195AE70023F4
:10AF0000F6E70B20002E00D02EE70722EB683A80F0
:10AF10001A7822705A7862705A88A2705A88120A77
:10AF2000E2701A792271DA886271DB881B0AA371D8
:10AF300075E7C046042900000228000000D8FFFF82
:10AF4000FFD6FFFF03280000FFFF000090BF0011A5
:10AF5000F0B58DB06B460020089120229B5E8342A5
:10AF60003DDAA64B187800F0A3FC071E32D0037818
:10AF7000B02B2CD10079023816281FD800F0B8FB6E
:10AF800017001E001E001E0031001E0096001E004D
:10AF90001D011E0052011E0073011E00CD011E0086
:10AFA00050021E001E001E008E021E00E302944B83
:10AFB00094491B8878880B80FBF72CF83800FCF745
:10AFC000ADFF914B1B68002B01D03800984738002B
:10AFD00000F066FD8020089B0002434018000DB081
:10AFE000F0BDEE220021874800F0A2FC0BAA3B7BBB
:10AFF0007989388900923A000D32FCF7B1FD0400DE
:10B00000804B1B78002C3FD146E0804B788805931D
:10B010007F4B4100CB5A0BAE073BDBB23288029329
:10B02000002301937B4B210006930093059BFFF7C0
:10B030006FFE744D002810D1069B3A8A1B889A42F5
:10B040000BD138000599123000F062FE002804D0C0
:10B050002B7862899B00EB185A80162306A81B18D0
:10B06000328820007989FCF7D7FE2B7804009A00FB
:10B07000AA1851880029C3D00133DBB22B700028F5
:10B0800007D006A9C98A9180634A12889A42BCD81F
:10B0900002E0012149429180002B04D0594978886F
:10B0A000FAF7ECFF8AE73E890A2479E000253E8919
:10B0B000574B06937B88069A5B009B5A033B9D4245
:10B0C00002DB002DF0D05BE0162206A812183B7BB5
:10B0D000798900923A0030000D32FCF741FD05906D
:10B0E000002858D04689017A7888FCF703FD041EB1
:10B0F00044D1464B78880793069B4100C95A454B7B
:10B100000439C9B206AAD28A069302910194009327
:10B110000599079BFFF7FCFD041E2FD1069B3949BB
:10B120001A88931C002D26D14B807988384B490012
:10B13000CB5A5119033B8B4220DD059B31485B897B
:10B1400041190B71A91C0135C9B2EDB20591451920
:10B150001B0A2B71059B2D490433181800F038FB8E
:10B160002C4B059A1B88D318DDB22C4B9E4205D080
:10B170000136B6B29CE749889942D6D0002D0CD052
:10B18000204C2800618800F033FD20702100788871
:10B19000FAF784FF12E7059CF0E7002C00D183E763
:10B1A0007B78142B00D109E716493B794E800B7050
:10B1B0000C717888FAF724FF00E7162406ABE41830
:10B1C00021003889FCF7B4FD011E00D1B7E1788871
:10B1D00022880F4C45002C5B0A4D013CE4B20294DE
:10B1E00000240F4B01940095FFF792FD041E00D040
:10B1F00014E129007888FAF761FFDFE6006BFF1F92
:10B20000B842FF1F1868FF1F0C68FF1F0C69FF1F63
:10B210004864FF1FFC69FF1FB642FF1FFFFF0000CD
:10B220001A68FF1F162406ABE41821003889FCF7C2
:10B230007FFD011E00D182E178882288AE4C450056
:10B240002C5BAE4D013CE4B202947C89AC4B019482
:10B250000095FFF75DFD041E00D0DFE0290078882F
:10B26000FAF736FFAAE60025A44B1D803B00F63313
:10B270001B78A24A78880792AB4208D99E4B128865
:10B280000693069943005B5A013B9A4203DB0799F8
:10B29000FAF728FF92E616246B00FB18059306AB1D
:10B2A000E418059B21001889FCF742FD011E03D11B
:10B2B000059B01241E8973E77888924B2288069C9F
:10B2C000099343001B5B904E013BDBB202930023CA
:10B2D00000960193099BFFF71BFD041E02D0059BFE
:10B2E0001E895DE77B88069A5B009B5A079A108847
:10B2F00032881218934202DC1B1A013B33807F4CC8
:10B30000023032880999001900F062FA23883288E5
:10B3100001359B182380EDB2A8E70BAA3B7B798906
:10B32000388900923A000D32FCF71AFC002505908E
:10B33000059B002B04D10A24002D00D16EE060E0B3
:10B34000059B7888197AFCF7D5FB0100041E63D1B0
:10B35000694C6C4B788806940993069B4400E45A28
:10B36000694B063CE4B20BAE32880793029401911C
:10B3700000930599099BFFF7CBFC041E4CD1079B5A
:10B380005E491B881A1D002D30D14A80059B5B4CFD
:10B390005A8963191A716B1C9BB2E318120A1A714D
:10B3A000162306A832881B1879890598FCF734FD06
:10B3B000FF21AA1C2E1D03350B00059092B2B6B2D8
:10B3C000ADB2002803D006ABDB8AD9B21B0AA218A3
:10B3D000651911712B714C4D301D2A88494920186F
:10B3E00000F0F6F92B88F618B5B2A1E7498891422A
:10B3F00007D17A8806995200525AEB18053A9A42B8
:10B40000C4DC3E4C2800618800F00AFB207021005B
:10B410007888FAF771FED1E5002DF2D13E89BFE6BA
:10B42000162606ABF61831003889FCF781FC3D0082
:10B430000400FA3500282DD0037A9B060CD4002294
:10B440007B893989788800923A000C32FFF7E8FB53
:10B45000041E10D03E8915E03088FFF741FB00281C
:10B460001AD08368002B17D02100122278889847C1
:10B47000041EE4D0EEE72B78002B02D17888FAF78F
:10B480004BFE00262B78002B00D097E5002C00D136
:10B4900094E585E60124DDE70E24DBE7162506ABFF
:10B4A000ED1829003889FCF743FC041E47D0037AC5
:10B4B0009B0611D4154A7B881188994203D0144801
:10B4C000814207D11380134BF2261D780023D9B295
:10B4D000A94221D30924A1E72888FFF701FB00280E
:10B4E0002FD08368002B2CD0210012227888984717
:10B4F000041EDFD092E7C0464864FF1F1868FF1F94
:10B500001A68FF1F0C69FF1FFC69FF1FF86AFF1F05
:10B51000FFFF0000F66AFF1F3100594354680133F2
:10B520006018615A0029D2D13C0008342100F2226F
:10B5300000F04EF921007888FAF7F6FD3EE5012487
:10B540006CE70E246AE71D4B1A887B889A4231D03B
:10B550007888FAF7F3FD31E5F22305985168434303
:10B56000CD18C95A00291FD03B7A012B0BD16C880A
:10B57000AB887888AA1D0094FFF752FB041E02D006
:10B5800000233B722E88F2220021280000F0D0F91F
:10B5900000232B80059B0133DBB20593084B0599F3
:10B5A0001B78064A8B42D7D801235B421380002CBC
:10B5B000CED0F5E5002634000596EFE7F86AFF1FC8
:10B5C000F66AFF1F70B504000E001500FFF796FA2B
:10B5D000031E08D131000548FFF790FA030011203F
:10B5E000002B02D01C8000209D7070BDFFFF00006A
:10B5F000F8B50B4F06003B780D001400FF2B0ED062
:10B600000A2000F005FB011E09D0B12303800023AE
:10B6100046800371C5800481387800F031FBF8BDA5
:10B620000D44FF1FF7B50F0008A90600088809A9F7
:10B630000B240988002821D10234022B1ED1557811
:10B6400013782D021D432B008B4301937334002B81
:10B6500014D1FB68300019000093FFF74FFB019CE9
:10B6600085420BD02A0030000099FFF7ABFF041E83
:10B6700004D12A0030007989FFF7BAFF2000FEBD0F
:10B68000F0B50E7885B003900AA805880120022E37
:10B690000DD14C682778647824023C43054FBC42A6
:10B6A00005D10398DBB201960095FFF7BBFF05B00B
:10B6B000F0BDC04602290000034B10B51B68002BEB
:10B6C00000D09847FEE7C046046BFF1F07B501A8EE
:10B6D000FFF7F2FF044A05480021121A00F0F8FAB9
:10B6E000F8F7CAF8FEE7C046086BFF1F1044FF1FBB
:10B6F00001B40248844601BC604700BF353BFF1FD0
:10B7000001B40248844601BC604700BF6571010076
:10B7100001B40248844601BC604700BF311B0000F1
:10B7200001B40248844601BC604700BF4D36FF1F8C
:10B7300001B40248844601BC604700BF055E0000BA
:10B7400001B40248844601BC604700BFD932FF1FE4
:10B7500001B40248844601BC604700BFB54C0100FB
:10B7600001B40248844601BC604700BFB132FF1FEC
:10B7700001B40248844601BC604700BF9D3AFF1FE8
:10B7800001B40248844601BC604700BF7130FF1F0E
:10B7900001B40248844601BC604700BF091B000099
:10B7A00001B40248844601BC604700BF3D4B010024
:10B7B00001B40248844601BC604700BFC56D01006A
:10B7C00001B40248844601BC604700BF213BFF1F13
:10B7D00001B40248844601BC604700BFE94C010047
:10B7E00001B40248844601BC604700BFF537FF1F23
:10B7F00001B40248844601BC604700BF1131FF1FFD
:10B8000001B40248844601BC604700BF056A0000DD
:10B8100001B40248844601BC604700BFB352010036
:10B8200001B40248844601BC604700BFE5480000FF
:10B8300001B40248844601BC604700BF350E0000D9
:10B8400001B40248844601BC604700BF4D1F0000A0
:10B8500001B40248844601BC604700BFC93AFF1FDB
:10B8600001B40248844601BC604700BF0919FF1FAC
:10B8700001B40248844601BC604700BF156B01005B
:10B8800001B40248844601BC604700BF911BFF1F02
:10B8900001B40248844601BC604700BF7539FF1FF0
:10B8A00001B40248844601BC604700BF2146010044
:10B8B00001B40248844601BC604700BFF54E010058
:10B8C00001B40248844601BC604700BFF94C010046
:10B8D00001B40248844601BC604700BF51470100E3
:10B8E00001B40248844601BC604700BF29510100F1
:10B8F00001B40248844601BC604700BFF13AFF1F13
:10B9000001B40248844601BC604700BF3519FF1FDF
:10B9100001B40248844601BC604700BF291C0000F6
:10B9200001B40248844601BC604700BF014C0100DD
:10B9300001B40248844601BC604700BF154D0100B8
:10B9400001B40248844601BC604700BF3555000081
:10B9500001B40248844601BC604700BF213AFF1F82
:10B9600001B40248844601BC604700BFE1170000F3
:10B9700001B40248844601BC604700BFDD66010097
:10B9800001B40248844601BC604700BFB539FF1FBF
:10B9900001B40248844601BC604700BFC9260000CC
:10B9A00001B40248844601BC604700BF554901000C
:10B9B00001B40248844601BC604700BF1D4B010032
:10B9C00001B40248844601BC604700BF3D18000036
:10B9D00001B40248844601BC604700BFF30E00007A
:10B9E00001B40248844601BC604700BF2124000026
:10B9F00001B40248844601BC604700BF0D520100FB
:10BA000001B40248844601BC604700BF810E0000BB
:10BA100001B40248844601BC604700BF4137FF1FA4
:10BA200001B40248844601BC604700BF090E000013
:10BA300001B40248844601BC604700BF595201006E
:10BA400001B40248844601BC604700BF456B010059
:10BA500001B40248844601BC604700BFA54F010005
:10BA600001B40248844601BC604700BFB14E0000EB
:10BA700001B40248844601BC604700BF017F00005A
:10BA800001B40248844601BC604700BF090E0000B3
:10BA900001B40248844601BC604700BF8930FF1FE3
:10BAA00001B40248844601BC604700BF434D010019
:10BAB00001B40248844601BC604700BFC94A010086
:10BAC00001B40248844601BC604700BF4136FF1FF5
:10BAD00001B40248844601BC604700BFEDA50000E8
:10BAE00001B40248844601BC604700BFA94601007A
:10BAF00001B40248844601BC604700BF0124000035
:10BB000001B40248844601BC604700BFD949010026
:10BB100001B40248844601BC604700BFADAE0000DE
:10BB200001B40248844601BC604700BF4551010092
:10BB300001B40248844601BC604700BFED4A0100E1
:10BB400001B40248844601BC604700BF75A90000EB
:10BB500001B40248844601BC604700BF312EFF1F7C
:10BB600001B40248844601BC604700BFDD520100B9
:10BB700001B40248844601BC604700BFC9A9000067
:10BB800001B40248844601BC604700BF252600007E
:10BB900001B40248844601BC604700BF85520100E1
:10BBA00001B40248844601BC604700BF1147010050
:10BBB00001B40248844601BC604700BFE928000088
:10BBC00001B40248844601BC604700BF7136FF1FC4
:10BBD00001B40248844601BC604700BFC521000093
:10BBE00001B40248844601BC604700BFFD38FF1F16
:10BBF00001B40248844601BC604700BF350E000016
:10BC000001B40248844601BC604700BF6DBC00001F
:10BC100001B40248844601BC604700BF1D4D0100CD
:10BC200001B40248844601BC604700BF691F0000A0
:10BC300001B40248844601BC604700BFC51D000036
:10BC400001B40248844601BC604700BF851F000064
:10BC500001B40248844601BC604700BF3539FF1F6C
:10BC600001B40248844601BC604700BFE938FF1FA9
:10BC700001B40248844601BC604700BF8B520100FA
:10BC800001B40248844601BC604700BF594F01001F
:10BC900001B40248844601BC604700BF0D3BFF1F52
:10BCA00001B40248844601BC604700BF9DA9000062
:10BCB00001B40248844601BC604700BF4550000003
:10BCC00001B40248844601BC604700BF5D17000014
:10BCD00001B40248844601BC604700BFB70E0000B3
:10BCE00001B40248844601BC604700BF79180000D7
:10BCF00001B40248844601BC604700BF55220000E1
:10BD000001B40248844601BC604700BF0934FF1FEC
:10BD100001B40248844601BC604700BFCD4C01001D
:10BD200001B40248844601BC604700BFD91B000033
:10BD300001B40248844601BC604700BF8D12000078
:10BD400001B40248844601BC604700BF5125000091
:10BD500000030102020303030403050006020700B7
:10BD6000080209030A030B030C000D000E030F0366
:10BD7000100311031303140315021602253C0011CE
:10BD8000593C0011000000000200000092BD0011AB
:10BD9000192A0F180A000000F1590000FD240000C4
:10BDA000414601006D81001181A10011D57500117E
:10BDB000717F00111954001151AF0011655000112D
:10BDC000353E0011653F001100000000161600000E
:10BDD00002000000DCBD0011F4FFF3FFD2FC000004
:10BDE000A5400011000000000000000054757961BA
:10BDF0000042312E39003030314100676974687576
:10BE0000622E636F6D2F707676780054484233004F
:10BE10000200000024BE0011292A282A272A262AE7
:10BE2000252A242A0A180000E204000071020000FA
:10BE300078EC0000050000007440000010270000AE
:10BE400060F000000400000006640000204E0000C6
:10BE500000000000060000005C4400001027000005
:10BE60006CEE000007000000050000001F501D00E0
:10BE7000023CB40000011A0019000000A1020000F9
:10BE80003031323334353637383941424344454610
:10BE9000000000001D580011715800110000000042
:10BEA00002000000ACBE00116F2A6E2A1A18EAD8F0
:10BEB000BC80F0FC600000000000000000005F0695
:10BEC0006B2F363D7D077F3F777C596E797100007F
:10BED00001A00000000000006410B71DC8206E3BE8
:10BEE000AC30D9269041DC76F4516B6B5861B24D81
:10BEF0003C7105502083B8ED44930FF0E8A3D6D6EB
:10BF00008CB361CBB0C2649BD4D2D38678E20AA052
:10BF10001CF2BDBDFB349B5F800000800010000060
:10BF200000000000D761001161780011FB61001171
:10BF3000697C00117F6200113F7C0011F5620011E5
:10BF4000157C001147630011DD7D0011AF63001106
:10BF5000DD7D0011E1630011977D0011F562001194
:10BF6000CD7B00116D630011757D00110000000094
:10BF70000000000053640011757D0011B5640011CC
:10BF800079780011052A042A012A002A02290328A7
:10BF9000012800280118001800000000000000001F
:10BFA00000000000000000870101020102010102FF
:10BFB0000102030304010301010101010303020162
:10BFC00003000D000E001000110013001401070102
:10BFD00008010A010B011C011D02040205020702EF
:10BFE000080219021A021C021D03010302031700B2
:10BFF0000201000504000807000B0A001716001DC7
:10C000001C010201010504010E0D011110011413A0
:10C01000011716011A19020201020B0A020E0D0283
:10C020001110021413021716030504030807030B6B
:10C030000A030E0D0001020307090A0B0E0F10116F
:10C0400012141718191A1B1F2021220099A8001179
:10C0500055A90011000000000200000096BF001169
:10C060000000000081B60011000000000200000086
:04C0700094BF001168
:020000041FFFDC
:10000000000000009D3D001198BD001194BD00113D
:100010004061FF1F00000000000000000000000021
:1000200000000000000000000000000000000000D0
:1000300000000000000000000000000000000000C0
:1000400000000000000000000000000000000000B0
:1000500000000000000000000000000000000000A0
:100060000000000000000000000000000000000090
:100070000000000000000000000000000000000080
:100080000000000000000000000000000000000070
:100090000000000000000000000000000000000060
:1000A0000000000000000000000000000000000050
:1000B0000000000000000000000000000000000040
:1000C0000000000000000000000000000000000030
:1000D0000000000000000000000000000000000020
:1000E0000000000000000000000000000000000010
:1000F0000000000000000000000000000000000000
:1001000000000000000000000000000000000000EF
:1001100000000000000000000000000000000000DF
:1001200000000000000000000000000000000000CF
:1001300000000000000000000000000000000000BF
:1001400000000000000000000000000000000000AF
:10015000000000000000000000000000000000009F
:10016000000000000000000000000000000000008F
:10017000000000000000000000000000000000007F
:10018000000000000000000000000000000000006F
:10019000FD32FF1F5D31FF1FC1660100000000003E
:1001A000000000000000000000000000000000004F
:1001B000000000000000000000000000000000003F
:1001C000000000000000000000000000000000002F
:1001D000000000000000000000000000000000001F
:1001E000000000000000000000000000000000000F
:1001F00000000000000000000000000000000000FF
:1002000000000000000000000000000000000000EE
:1002100000000000000000000000000000000000DE
:1002200000000000000000000000000000000000CE
:1002300000000000000000000000000000000000BE
:1002400000000000000000000000000000000000AE
:10025000000000000000000000000000000000009E
:10026000000000000000000000000000000000008E
:10027000000000000000000000000000000000007E
:10028000000000000000000000000000000000006E
:10029000000000000000000000000000000000005E
:1002A000000000000000000000000000000000004E
:1002B000000000000000000000000000000000003E
:1002C000000000000000000000000000000000002E
:1002D000000000000000000000000000000000001E
:1002E000000000000000000000000000000000000E
:1002F00000000000000000000000000000000000FE
:1003000000000000000000000000000000000000ED
:1003100000000000000000000000000000000000DD
:1003200000000000000000000000000000000000CD
:1003300000000000000000000000000000000000BD
:1003400000000000000000000000000000000000AD
:10035000000000000000000000000000000000009D
:10036000000000000000000000000000000000008D
:10037000CDB60011000000000000000000000000E9
:10038000000000000000000000000000000000006D
:10039000000000000000000000000000000000005D
:1003A000000000000000000000000000111BFF1F03
:1003B000000000000000000000000000000000003D
:1003C000000000000000000000000000000000002D
:1003D000000000000000000000000000000000001D
:1003E000000000000000000000000000000000000D
:1003F00000000000000000000000000000000000FD
:08183800106FFF1F4118FF1F94
:10184000024981F3088802F0DFF90000106FFF1FE2
:1018500070B500241E491F4A1F484C6308CA1B0567
:101860001B0DE4188242F9D11C4B80228B630021AE
:1018700009201B4B920519621A4B1B4DDA671B4B53
:10188000DA688243DA609A68194802409A60112047
:10189000296002F08FF8112002F06CF86B6C154A89
:1018A000112013406B64EE23DB006343124A1B0CD0
:1018B00013840122114B9A7201F006FC104B1B7825
:1018C000002B04D10F4B1021187802F065FB70BD7E
:1018D000000005400806054080060540FF010000A5
:1018E00000F0004004E100E0003800403CF000401F
:1018F000FFDFFFFFFFFEFFFF1061FF1FC461FF1F3F
:10190000F263FF1FF061FF1F10B502F05DFB0728B7
:1019100004D0122808D0022808D010BD044A0420A0
:10192000136B01331363F8E70220F6E71420F4E7A2
:10193000F064FF1FF8B507000C00260025005036A4
:1019400030785135002804D10300287058342370B2
:10195000F8BD2978CA00481E8141A3183800A25C4E
:101960005B68C9B2FFF7D0FF00280DD12B78DA00F1
:10197000A218013350602B703378044A013B337056
:10198000136A01331362D8E70123DFE7F064FF1F16
:101990005C234343074910B5C9180B0058331B7823
:1019A000012B05D1FFF7C6FF034A936A0133936207
:1019B00010BDC0462465FF1FF064FF1F10B502F084
:1019C00013FB064A0121130010CB4942D967044B8F
:1019D000136002F051FA200010BDC04600E100E0A3
:1019E0001000100010B5040002F0FEFA024B1C605B
:1019F00002F042FA10BDC04600E100E0431E5A4228
:101A00005341A022F0B5D2015B421340154D164A56
:101A100040019B182A18127E8BB00191002A1BD01E
:101A20001A000832D46F0022E6B206AFE4B2944244
:101A30000EDC2818C369002B08D0019902AA117185
:101A400006AA049202AA167303A898470BB0F0BD29
:101A50001978B9540132EAE71A7D1A7806AB0126E3
:101A60001A70E6E7B067FF1F00400040F0B5254B55
:101A700004004001C25C85B0002A2BD01A18117EE8
:101A8000002927D0917E002924D01179022921D163
:101A90001689D788D168F51BADB22A1C102D00D944
:101AA000102292B2BE4217D11818012303710023ED
:101AB000C269C38003819A4206D06846032103733A
:101AC0000171029301A890470820002C00D0192032
:101AD00001F0FAFA05B0F0BD013C65426C41A02569
:101AE0006442ED012C40084D1B186419074D063364
:101AF000013A92B2AA42EDD01888461C1E80085CBA
:101B00002070F5E7B067FF1F00400040FFFF0000B6
:101B10000F220E4B10B59868104002380A280BD8D7
:101B200001F0FEFF0D0A0B0A0A110A0A0A0A060052
:101B300002210020FFF762FF10BD0121F9E700201C
:101B4000FFF794FFF8E7DB6FF6E7C0460040004080
:101B50000F220E4B10B59868104002380A280BD897
:101B600001F0DEFF0E0A0B0A0A120A0A0A0A060030
:101B700002210120FFF742FF10BD01210800F9E713
:101B80000120FFF773FFF7E7DB6FF5E700900040F8
:101B900013B5334C2378072B3DD8324B1A78324B90
:101BA000002A39D18022196852020A431A6025207E
:101BB00001F0C0FE20232D4A11680B4380211360E1
:101BC0006B460422C90508680733104228D08021DB
:101BD0000422C905C86810422ED080212020C905E2
:101BE000CA688243CA6014221A701A78002A2FD158
:101BF0008021C905C86820320243CA6014221A70C5
:101C00001A78002A28D11A4B1A7D22785A601D2290
:101C10001A705932DA6013BD1A6816490A40C5E7CE
:101C2000086802430A6014221A701A78002ACED07B
:101C30001A78013AD2B2F7E7C8680243CA601422A0
:101C40001A7019784A1ED2B21A700029F9D1C4E765
:101C50001A78013AD2B2C7E71A78013AD2B2CEE77F
:101C60004843FF1F1044FF1F3CF000404043FF1F4C
:101C700000200040FFFFFEFF564B70B51B68012B94
:101C800003D1554A936D0133936502F035F8534BF8
:101C9000534A1860534B544C1A600123534A136043
:101CA000534A13602378002B06D00622514952482C
:101CB00001F0A2FF00232370504A514B10681B789B
:101CC000C1B2002B0ED14F4CC0B223785BB2002BB7
:101CD0004FDB237824785BB264B21B0424021B1907
:101CE0001B1813600B1C50294ED95023464A4749F4
:101CF0001078DBB2FF2202284BD10868444C454DD6
:101D0000267890432A78964254D9227824782E78DF
:101D1000023B5D10A31B6B435201D31A10335B11BE
:101D20001843086002F040F8031F012B45D83A4BD6
:101D30001B78002B06D0394B1B78002B02D00020DB
:101D400002F0EAF8A122364B92009978354B4A43CB
:101D50001B689B18832292009B181B78033B012B66
:101D600003D8AF20400001F057FF01222E4BDA824A
:101D700070BD237824785BB264B2FF33FF341B0458
:101D800024021B190138ABE7CAB2022AAED20223E1
:101D9000ACE70868254C264D267890432A78964271
:101DA00008D9227824782D78023B5B10641B6343AA
:101DB0005201B2E72378DBB2B2E70228D5D11D4B3E
:101DC0001B78013B022B03D91B4B1B78022BCCD178
:101DD0006C20C8E79809FF1FFC0FFF1F3C64FF1F22
:101DE000FF3F0000141003404064FF1F0C1003402D
:101DF00000100340D50BFF1F7211FF1FB4000340FA
:101E00008C09FF1F680AFF1F490AFF1F9400034047
:101E1000460AFF1F470AFF1FF908FF1F2209FF1F7D
:101E2000300DFF1F3409FF1FBC0BFF1F440AFF1FAB
:101E3000450AFF1F1C09FF1F2309FF1F10B502F0F1
:101E4000BBF80022014B1A8010BDC0463A64FF1F48
:101E500010B502F0C1F8A121054A89009478054A1D
:101E600061431268044B5218528C1A8010BDC04650
:101E7000300DFF1F3409FF1F3A64FF1F10B50D4BD3
:101E80000D4A9978A1239B004B431268D218531D29
:101E9000D97F0A4B1B88994209D2441C07D0C82815
:101EA00005D0D2695B1A5A43054B5343C01801F061
:101EB00053FE10BD300DFF1F3409FF1F3A64FF1F92
:101EC0007102000070B5244D2B68002B28D001F062
:101ED00003FF2B68D8402B680400002B27D001F0AB
:101EE00073FE2B68D8401D4B1D4A9978A1239B0097
:101EF0004B431268D118D25C91239B00002A20D05A
:101F0000CA580132CA50174B17491B6808688342E8
:101F100014D3D23B181A012A1AD0144B186070BD82
:101F200001F0DAFE124B196801F0B6FED3E701F0BA
:101F30004BFE0F4B196801F0AFFED4E70D495B185B
:101F4000E8E7CA500C4B1B68DB68E418201AE4E78A
:101F5000F530FF30E1E7C0461C08FF1F300DFF1FC2
:101F60003409FF1F9C09FF1F3C64FF1FA009FF1FCE
:101F70001808FF1F2DFF3F004464FF1F70B50400C9
:101F80000D00282916D10300A433C2881B889B1A90
:101F90000B4A9BB293420DD906006A3605223100E6
:101FA000653001F0D1FE002804D13100200001F09D
:101FB000EBFE70BD2900200002F03EF8F9E7C046B4
:101FC000FE7F0000F8B50500012002F01DF8134C5B
:101FD000A36AA26A9342FBD1114E336001F0C4FFA1
:101FE0001049030008601048426894460F4A176879
:101FF0000022BC4501D24268BA1A0D48026032681C
:10200000AD18A422E562606A520302436262094A83
:102010001278002A01D00F3B0B60F8BD00F00040A1
:10202000340AFF1FE408FF1F28100040180AFF1F92
:102030001C0AFF1F1C09FF1F70B580241025E40532
:10204000A3682B43A36001F007FFA368AB43A36021
:1020500070BD0000F7B5160080221C001023D205C9
:102060000191916805000B43936000225A4BD730D1
:102070001A6001F059FE9D232A002F009B00EB58A7
:10208000CA3201210092FC37002B01D00021009AB6
:10209000386801F0C9FE2900009BCB311A784F4BFC
:1020A000D3351A604B780A781B0213438A781204DE
:1020B0001A43CB781B061343494A1BBA13604B796A
:1020C0000A791B0213438A7912041A43CB7931002F
:1020D0001B061343434A1BBA13606B782A781B0212
:1020E0001343AA7812041A43EB781B0613433E4AA3
:1020F0001BBA1360019A330213433C4A13603C4BF2
:1021000022001B1B9C4603293DDCB3089A001300E8
:102110005142B21A032A46D1354AE018511A827840
:102120004078120400020243E05C043302430A6078
:102130000022FF2B4BDDF0222E4B12011A600F22E2
:102140002D4B1A602D4A1368002BFCD00023224A25
:1021500027491360091B321D0B191B68043A180A22
:1021600023706070180C1B0EA070E3700434002AFA
:10217000F2DC802210213B68D20501333B6093687A
:102180008B439360F7BD6346D578981893782D06F6
:102190001B042B43157804392B43557804322D0248
:1021A0002B430360AFE7022A0AD1114AE05C511ABF
:1021B000E2185278120202430A6004339BB2B7E776
:1021C000012AB5D10A4A521AE15C1160F5E70849C3
:1021D00059180A600433ACE7000004403C00044096
:1021E0003800044034000440300004400C00044037
:1021F00000010440040004401000044014000440A6
:10220000F7B5150080221C001023D20500919168BB
:1022100007000B4393600023654AD730136001F039
:1022200083FD9D233E009B00F9583B00CA363200D7
:10223000FC33002900D07FE0586801F0F5FD39003B
:1022400032785C4BCB311A604B780A781B0213430F
:102250008A78AC4612041A43CB78281D1B06134318
:10226000554A1BBA13604B790A791B0213438A79CA
:1022700012041A43CB791B061343504A1BBA13604E
:102280004B7A0A7A1B0213438A7A12041A43CB7AD6
:1022900021001B0613434A4A1BBA1360009A2B0203
:1022A0001343484A13602200474B1B1B0093009BBB
:1022B000CE785B1801938B7836061B0433430E7877
:1022C000043833434E78043136023343019E336081
:1022D0000328ECDC0321A808431C9B002940800054
:1022E00003292BD13849E5185E18A9786D78E35C8D
:1022F00009042D02294319433160030008330021EA
:10230000FF2B2DDD314B324919600F21314B196004
:10231000012327490B60304B19680029FCD00621A6
:102320001B680B40042B20D080220020D20593682C
:102330000A318B439360FEBD01217DE7022908D15C
:1023400021495D18E1184978E35C090219432960C5
:10235000D3E70129D3D11C495918E35C0B60CCE7C2
:102360001948181801600433CAE7002310490B60AC
:102370006346002B0CDC3B00FC335A681021013211
:102380005A608022D205936801208B439360D2E784
:10239000009B9B181B68190A13705170190C1B0EB7
:1023A000D37004235B4291709C440432E0E7C04642
:1023B000000004403C000440380004403400044065
:1023C000300004400C0004400001044004000440BC
:1023D000080F0000100004401400044070B5061EF1
:1023E00019D002225A4B9B799343012B13D1594B9D
:1023F0001A78FF2A0FD15A78FF2A0CD19A78FF2A2F
:1024000009D1DA78FF2A06D11A79FF2A03D15B793C
:10241000FF2B00D199E0504B0C201A78012A08D0EC
:1024200000224E4D1A7029780B00093B042B01D86D
:10243000212070BD4B1F012BFAD9454CA37B042BE7
:1024400000D982E0A279032A00D97EE09A1ED2B296
:10245000012A02D860881F2877D9002E56D0012E75
:1024600073D1A0880128E3D0002907D1581E032882
:1024700003D801F055FB121715122E702978481E4B
:10248000032811D80025364B1D602823237501F041
:1024900093FCA84227D0A580CAE702212970EDE766
:1024A0000421FBE70321F9E707390129C0D82D49A9
:1024B0000968C96A8906BBD52B4908780028B7D1B5
:1024C000012A01D9002BB3D102230B708021274DA3
:1024D000263389012878237501F05EFB8021287856
:1024E000890101F059FD0123A380214B1B78002BAA
:1024F0000AD0FA2280211F4B92001B8809025A43FE
:102500001A4B187801F0E8FC002092E701F06CFD0E
:102510002B78A680073B012B03D917482E7001F0BA
:102520008BFC114B114C1A78002A06D08021002216
:10253000207889011A7001F02FFB01F09DFC8021A9
:102540002078090201F028FBDEE7122071E7C0467F
:10255000A60BFF1F6B09FF1F1A09FF1F1C09FF1F96
:102560004809FF1F4464FF1F2309FF1F1B09FF1FAA
:102570002109FF1F2C09FF1F0010004010B5002982
:1025800001D001F0F9FB10BDF7B5604B01919978CE
:10259000A1239B004B435E4A060014681022E418F6
:1025A000D6235B00E0583623FF33E35C00279343D8
:1025B000222B41D1574B0F3A1A600760012501F0D9
:1025C000F3FA019B1880E8235B00E35C002B01D049
:1025D000B34258DD0023504FFB70AD33FF33E35857
:1025E0001A68002A03D09B88DB439B071DD0382341
:1025F000FF33E35C002B18D09B235B00E35C002BD4
:1026000013D1D133FF33E35CB3420EDAA4235B0072
:10261000E15AE018090A023101F0E6FB2300012229
:10262000FE33013E01351A87FA70E8235B00E35C54
:10263000002B2AD0A8B2FEBD03683D00002BBED0FF
:1026400081880430090A023101F0CEFBD6235B00F9
:10265000E3581F60B2E72300B133BA00FF33985844
:10266000013781880430090A023101F0BDFBE823FB
:102670005B00E35CBB42EEDCE822F61AED180023B7
:102680005200A354A6E70027F1E7200001F01CFC4C
:1026900000281FD0002E1DDD7319882647190193CD
:1026A000B600200001F0D0FB5A30800020184068AE
:1026B000013581880430090A023101F095FB2000C0
:1026C00001F012FBA3590133A351BD4202D0019B7B
:1026D0009D42E6D1114BE35C002BABD095239B00D0
:1026E000E35C002BA6D00E4BE15A0029A2D00D4A84
:1026F000A35C994202D90133A3549BE700231A211A
:102700002000A35401F008FB94E7C046300DFF1FE2
:102710003409FF1F00140340E010FF1F5A0200009D
:10272000720200005E0200000D4970B54A6E0D4C49
:10273000D2038B69D20BA24206D80B4D0224AA42C7
:1027400004D901F019FA70BD02246442E2181500A0
:102750007E2425402242F4D0A3432B438B61F0E733
:1027600000F000400A200000FC1C0000F8B51D4BE2
:102770001D4F1A78002A10D1BA7B002A02D10132EB
:102780001A7003E0032AFAD0022AF8D001F014FBF1
:1027900000220120154B1A70F8BD154B154D1C6811
:1027A000154B9E7801232B702878C0B200F09EFB59
:1027B000BB7B002B0BD101F0CFFAA1239B0073430D
:1027C000E41883239B00E41823782B70E4E7032BA1
:1027D00002D101F021FBF0E70020022BDCD101F057
:1027E00043FAEAE71C09FF1FA60BFF1F2309FF1F7F
:1027F0003409FF1F490AFF1F300DFF1FF0B587B0D6
:102800000EAD2F780FAD2D780593AC4663461400BE
:102810000E4D0CAA12782E7803930D9B0092019313
:102820002200059B029701F05FFB2E70012C01D066
:10283000042C08D1802206498B889343054A1278DC
:10284000D20113438B8007B0F0BDC0461C09FF1FA7
:102850006C11FF1F7809FF1F0B001B3B70B50400B4
:102860003020E02B0DD81300E025493BFF3B9BB205
:10287000ED00AB4205D8034B200019825A8201F0CB
:102880007BFB70BD8410FF1F10B501F035FA054BBE
:1028900000205B68052B04D9034A5268D20200D499
:1028A000980810BD00100040FCE100E070B501F098
:1028B0009BFB0D4B1B68FC33DC691D6AFFF7E4FFD3
:1028C0006419844204D2094B01241B68002B07D0F1
:1028D00004220024064B1A70064A9369013393615F
:1028E00001F0CAFA200070BD4464FF1F9809FF1F61
:1028F0002309FF1FFC0FFF1F70B50C4D2B68FC3325
:102900005C6A01F071FBFFF7BFFF2B680025FC3309
:102910009B6AE318834204D2054B1B68AB4200D18B
:10292000051B01F0A9FA280070BDC0464464FF1FD2
:102930009809FF1FD722044B92009B5810B5002B1B
:1029400000D0984710BDC0460000FF1F10B501F031
:10295000CFF8FFF7EFFF2749274BCA6D274C1A40E6
:1029600084235B001343CB65254B1B68186A01F079
:102970004BFB244B244A1A60244B254A1A60A022A0
:10298000244B52001A60244B187801F005FA2000FD
:10299000224901F0B9FA0023A3600233A360204B5F
:1029A0002049236003232048A36001F0ADFA1022E0
:1029B0001E4BFF201A60802252031A60802292036D
:1029C0001A60802212041A6001F0A6FA012001F0B8
:1029D000DBF8FA20400001F017FA582001F01CF94A
:1029E000134801F0D1FA012001F0A6FA072001F006
:1029F000BBF810BD00F0004000FEFEFF14100040C8
:102A00004464FF1F000003400180063DBC000340FA
:102A100034080000A40003404A0AFF1F71020000AE
:102A2000C3090000FFFF3F002810004000E100E064
:102A300030750000674E336888331B6883F308885D
:102A400001F0C2F9644A6549136800200B40136025
:102A5000634B644A1B68934200D1A6E001F024F95D
:102A60000221614A13688B431360FFF76FFF5F4BCE
:102A70005F4C1878C0B201F017FA0023A36002334C
:102A8000A3605C4B0120236001F0BEFA0323A36026
:102A900001F04AFA040001F02FF9050001F044FAB0
:102AA000554B186001F0C8F8544B1968621A531E50
:102AB000A14200D213008022D203934201D39B0291
:102AC0009B0A3268D16AC90700D471E04C491C0CDA
:102AD00009689BB24C4359432402090A641803262F
:102AE0004849FC3293680A6847489B1A474A076876
:102AF000126847499B18474A9A1833409208DB19D5
:102B00000A600360042B03D9013233400A6003607A
:102B10000E684149A619300001F0BEF83F4F3E490A
:102B20003B68C3183B603000019301F0C5F83C4E90
:102B30003068081838493060884205D9019B013354
:102B40003B6001F0B9F8316001F0FEF9354B1B78BC
:102B5000002B0DD001F0D0F8334B621B196812180E
:102B60008A4232D24919091B091A304801F0CCF9BE
:102B70002F4E337A002B0ED001F0BEF8621BF168A5
:102B80001218914224D94919091B091A294801F040
:102B9000BBF900233372284B83F3088801F03CFA19
:102BA000002001F081F801F087F901F07DF85CE781
:102BB000DC0199000234641A5900641A09214B435C
:102BC0008033CB40A408E41889E7FA218900CCE7D8
:102BD0001A49DBE74464FF1F1CF00040FFFFC1FF00
:102BE0000C0AFF1FB641210310000040490AFF1FD5
:102BF00014100040C3090000100AFF1F340AFF1F11
:102C0000380AFF1F200AFF1F280AFF1F1C0AFF1F88
:102C1000240AFF1FC4090000710200006008FF1FA2
:102C20002C0AFF1F1C09FF1FE408FF1F00100040B3
:102C3000740BFF1F3C10004000000020DC0500006A
:102C4000A022054B92009B5810B5002B01D098474D
:102C500010BD01F081F9FBE70000FF1FA122054B29
:102C600092009B5810B5002B01D0984710BD01F081
:102C700073F9FBE70000FF1FA222054B92009B584F
:102C800010B5002B01D0984710BD01F065F9FBE7A6
:102C90000000FF1FA322054B92009B5810B5002B8C
:102CA00001D0984710BD01F057F9FBE70000FF1F66
:102CB000A422054B92009B5810B5002B01D09847D9
:102CC00010BD01F049F9FBE70000FF1F70B501F0EE
:102CD00013F84F4B186001F00FF90400C30702D43A
:102CE00001F08AF870BD00224A4B1A604A4B1878EE
:102CF0000138042829D800F013FF0320181C2400F1
:102D0000200001F001F80128ECD0444C2378042B7A
:102D10006ED101F049F90028E4D000F065FF582099
:102D200000F07AFF02232370DCE7200001F0B4F802
:102D3000E9E7200000F0A0FFE5E7200000F04CFFED
:102D4000E1E7200001F070F9DDE701F02DF8050062
:102D5000012808D1324B1B78053B012B03D82000FA
:102D6000FFF76EFFD1E72D4B1B78022B01D0052B0F
:102D700020D1022D28D12B4B9B7BAB431CD12000B3
:102D8000FFF76CFF264B18780128BED16405BCD430
:102D9000244925224B7B034205D1233A13405A4252
:102DA000534126331A000B7D9342AED9322001F0F5
:102DB00013F8AAE7022D07D1194B1B78052B11D167
:102DC0002000FFF759FFDDE7012D0BD1012B03D1C7
:102DD0002000FFF75FFF98E7062B03D12000FFF7E5
:102DE00067FF92E7200001F0B7F8022D8DD1C9E707
:102DF000032B04D10C4B987C00F02EFF72E7072BBD
:102E000000D06FE7094B987B01F03EF86AE7C046B7
:102E10009C09FF1F9809FF1F9009FF1F2309FF1F2F
:102E20001C09FF1FA60BFF1FBC0BFF1FD40BFF1FAE
:102E3000FA210A4B0A4A49001A640A4A5A500A4AB5
:102E400004395A50094A08319A64094A5A50094AC1
:102E50005C315A50084ADA667047C0460000FF1FCE
:102E6000FD27FF1FF928FF1FAD28FF1FDD23FF1FD0
:102E70006D27FF1F7D1EFF1F511EFF1FF7B50B0C97
:102E8000FF270122009300233C001E001D009446F2
:102E9000019089B262469A401000084018413618E5
:102EA000B6B2FF2F02D1012E00D19FB2009802408E
:102EB0001A41AD18ADB2FF2C02D1012D00D19CB248
:102EC0000133102BE6D10320012E07D1012D04D1AF
:102ED000019B2401E4191C700138FEBD102EFCD1A9
:102EE0000238102DF9D00230F7E700008023F7B543
:102EF0009C46264B264F01932649274A274D284CAE
:102F0000284B02281AD1604638600868264E3040A7
:102F1000802636033043086001990978002909D1D9
:102F20001660224A2A60224A2260E02219689143F0
:102F3000A03A1BE08021C9021160F2E766463E60BC
:102F40000F68194E3E408027FF023E430E600199F4
:102F5000097800290DD1176001280ED1154A2A6081
:102F6000154A2260E02219689143C03A0A431A6068
:102F7000F7BD802189021160EEE7E0210F4A02438C
:102F80002A600F4A22601A688A43F0E74B0AFF1F43
:102F9000E0000340D80003409000034000000340DD
:102FA0005000034040000340FFFFE3FF0280063D66
:102FB000804508220180063D806608220080069830
:102FC00080550822F8B51E4B80261A680020140090
:102FD0003440324232D11A681A4F32431A60012209
:102FE0003B68063093433B6001F00EF80122164D1A
:102FF0002B681E432E603B680A2613433B608027E4
:10300000BF00124B1B683B4211D1013EF6B2FF2EAE
:1030100009D17E220E4B1C682B68E40B14409343AD
:1030200023432B6005E0082000F0EEFFE9E7002EC7
:10303000EFD180222B68600893432B60F8BDC04617
:10304000C4F000405CF0004018F0004068F0004020
:1030500060F0004010B500F0E7FD01215820034A60
:1030600000F0CAFFFFF7AEFF10BDC046600AFF1FA9
:1030700010B578220021034800F076FE00F0F4FE3F
:10308000002010BD3867FF1F70B5040000F0ACFFD2
:1030900000230C200B4A010059438D18515C002974
:1030A0000DD0A14208D1012300246B7000F00CFE6A
:1030B00000F0E2FE200070BD01330A2BEBD1122498
:1030C000F6E7C0463867FF1F70B5040000F08CFFBC
:1030D000002319001D000D4A1078002806D0A042D8
:1030E0000CD1557001310C320A29F5D1002B0AD1CF
:1030F00000F0BAFE00F0C0FE002070BD5078461E01
:10310000B0411B18EEE700F0DFFDF3E73867FF1F63
:10311000F7B504000C20002384460E4D019267464B
:103120005F43E85D7E19A04212D000280BD10A4B04
:103130009C4662461B7808331370019B70707C5567
:103140007160B360FEBD01330A2BE8D10320F9E7BB
:103150000720F7E73867FF1F3467FF1F8020F8B5A7
:10316000484BC0051B68C1248360474BFF251A6884
:10317000012313434361454BA4001A68444B40218B
:103180001A60444B1A68444B1A60444B1A59AA43BC
:103190001A51C52292009E58AE4331438026995061
:1031A0009F583F49F6010F403E439E509E5880274E
:1031B0003602360A3043985080201A5900020A40DD
:1031C00002431A5104341A59364E3F0432408026C5
:1031D0003A431A511A5936061202120A32431A5148
:1031E00008341A5980260A4002431A51C322920019
:1031F0009F58B446AF4337439F509F58294E0F40C6
:1032000007439F509F583740802636043743802617
:103210009F509F5836063F023F0A37439F50C022B7
:103220001F59AF433A431A511A591202120A164350
:10323000C6221E5192009C58AC4365462C439C50BC
:103240009C5800250C4020439850C72080001A58F5
:10325000154C1140C02212020A431A50134B1B781E
:10326000DB08AB4201DC0020F8BD2378002B06D040
:10327000A368002B00D0984701350C34EEE71220EC
:10328000F2E7C0464443FF1F4043FF1FB0F0004039
:103290003067FF1FB4F000402C67FF1F00E100E023
:1032A000FF00FFFFFFFF00FF3867FF1F3467FF1FAE
:1032B000030010B51F2809D8072200201340072457
:1032C00004490A78A24313430B7010BD0023062063
:1032D000F5E7C0463467FF1F054B06491B780A68AF
:1032E00005485B0702401B0B134300200B6070472F
:1032F0003467FF1F1CF00040FFFFC1FF70B50C25B5
:10330000FFF7EAFF0A4B1C780A4BE4086543ED1807
:10331000002C01D1200070BD2B78002B06D06B68EB
:10332000002B00D09847013C0C3DF1E71220F2E75A
:103330003467FF1F2C67FF1F1FB5002102220B00FF
:1033400001910091052000F0F7FC02230B490A6867
:103350001A42FCD120230393039B5A1E0392002B95
:10336000FAD1074A1368002BFCDA0B246C442000C6
:10337000012100F021FC207804B010BD90C800406D
:1033800000C8004013B504000A4B0193019B002BB9
:1033900001D1112016BDFFF7CFFF230003400442E7
:1033A00005D0052000F030FE019B013BEDE7180041
:1033B000F0E7C046FFFFFF0707B500F015FE8022CB
:1033C0000821D205936A0191002B01D1073991623E
:1033D00002210C4A11600199481E01900029FAD17E
:1033E00003311160053101910199481E01900029B6
:1033F000FAD11160002B02D18022D205936200F035
:103400003BFD07BD00C00040F0B52D4C89B02378CE
:10341000002B4FD1FEF7D2FA02232A4F03903A68CD
:103420001A42FCD120230693069B5A1E0692002BBB
:10343000FAD1254E3368002BFCDA0120FFF7A2FFFA
:10344000011E02D0112009B0F0BD0300032201903B
:10345000009005AD9F2000F06FFC0321280000F0D4
:10346000ABFB02233A681A42FCD120230793079B47
:103470005A1E0792002BFAD13368002BFCDA012088
:10348000FFF780FF0028DDD10398FEF7ABFAAA789A
:103490006B7811041B020B4329780B436360130004
:1034A000113B0A49052B07D801239340A3600B6009
:1034B000012323700020C6E780231B03F6E7C046E4
:1034C0002C43FF1F90C8004000C800409808FF1F11
:1034D0001E4B30B55A6818781D4B85B0D318594229
:1034E0004B4101210093002300F0CEFB194B1A4AF7
:1034F00002259A6300221A6510325A658022C4217F
:103500009D65164B1648D202DA6789004258154B62
:1035100080241A4080231B0413434350642341201A
:103520000393E40500F006FA402000F003FA656218
:10353000039D6B1E0393002DFAD103236362FFF7F3
:103540003BFFA562FFF760FF05B030BD3843FF1FAA
:1035500095FFFEF700C80040050001FF04E100E010
:1035600000E100E0FFFF00FFF0B585B00700FEF7C7
:1035700025FA022305002D4C22681A42FCD1202393
:103580000093009B5A1E0092002BFAD1284E3368FC
:10359000002BFCDA0120FFF7F5FE002803D01124F0
:1035A000200005B0F0BD234B2360022322681A429D
:1035B000FCD120230193019B5A1E0192002BFAD1CA
:1035C0003368002BFCDA0120FFF7DCFE0028E6D18F
:1035D000194B1F60022322681A42FCD12023029358
:1035E000029B5A1E0292002BFAD13368002BFCDAA0
:1035F0000120FFF7C7FE0028D1D1104B2360022322
:1036000022681A42FCD120230393039B5A1E039283
:10361000002BFAD13368002BFCDA0120FFF7B2FE51
:10362000041EBCD12800FEF7DDF9B9E790C80040C0
:1036300000C8004001000006A8C800400180000149
:1036400010B50020FFF790FF10BD000010B5064B2D
:1036500018705960FFF73CFF00211320034AFFF761
:1036600057FD002010BDC0463843FF1FD134FF1F57
:10367000F0B5040085B003920291FEF79FF988220D
:1036800063035B0B52051A438023DB059D6A80238D
:10369000274F0092BA68002601901B039A420CD96A
:1036A000F82326001B041E401C4206D08022214B1A
:1036B00052025E6219680A431A60002D0BD100F0B5
:1036C00093FC02221C4B1A608023DB055A62013AEC
:1036D0009A6200F0D1FB0023039A934220D1002D7F
:1036E0000AD100F081FC144B03221D608023DB050E
:1036F0005A629D6200F0C0FB8023BA681B039A42A5
:1037000008D9002E06D000220A4B0C495A621A68CA
:103710000A401A600198FEF765F9002005B0F0BD77
:10372000009A0299D2181278CA540133D4E7C046DD
:103730002C43FF1F00C8004000C00040FFFFFEFFF9
:10374000F0B587B0029103920400FEF737F90190BB
:1037500000F04AFC802302250122234EDB05356060
:103760005D629A6200F088FB204F3B682B42FCD1DF
:1037700020230493049B5A1E0492002BFAD11C4D63
:103780002B68002BFCDA0120FFF7FCFD002802D09B
:10379000112007B0F0BD2000039A029900F054FAFE
:1037A000022304003A681A42FCD120230593059BAA
:1037B0005A1E0592002BFAD12B68002BFCDA01204F
:1037C000FFF7E0FD051EE3D100F00EFC802303228D
:1037D000DB0535605A629D6200F04EFB0198FEF7F2
:1037E00001F9E0B2D5E7C04600C0004090C80040F3
:1037F00000C80040F0B5802489B00600FEF7DEF86E
:10380000E405A36A02250393029000F0EDFB012377
:10381000304F3D606562A36200F02EFB2E4C2368A2
:103820002B42FCD120230593059B5A1E0592002BA9
:10383000FAD12A4D2B68002BFCDA0120FFF7A2FDFC
:10384000002803D01124200009B0F0BD244B2360D0
:10385000022322681A42FCD120230693069B5A1E9B
:103860000692002BFAD12B68002BFCDA0120FFF71F
:1038700089FD021EE6D11B4B03211E60030001904F
:103880000090202000F058FA022322681A42FCD14E
:1038900020230793079B5A1E0792002BFAD12B680F
:1038A000002BFCDA0320FFF76DFD041ECAD100F0E7
:1038B0009BFB80230322DB053C605A629C6200F084
:1038C000DBFA039B002B01D1FFF776FD0298FEF790
:1038D00089F8B8E700C0004090C8004000C8004028
:1038E0000100000694C8004007B5000201910422BF
:1038F000000A01A9FFF724FF0EBD000073B5050003
:1039000005240B4AA3005B429B1819686B46DE1D19
:103910003000FFF7B3FA022804D133782B55013C6D
:10392000EFD276BD052CFCD00128FAD10230F8E7A1
:10393000140900111F2807D8012380228340D205D3
:1039400091680B43936070473F2808D80123802279
:1039500020388340D20551690B435361F3E75F2858
:10396000F1D80123802240388340D205116A0B43ED
:103970001362E8E71F2807D8012280218240C90589
:103980008B6893438B6070473F2808D801228021C1
:1039900020388240C9054B6993434B61F3E75F28A8
:1039A000F1D80122802140388240C9050B6A934337
:1039B0000B62E8E71F2810D880230200DB05153AC8
:1039C0001968012A06D820229143196019680A4310
:1039D0001A60704701228240F6E73F2811D8802301
:1039E0000200DB05353AD968032A06D81022914334
:1039F000D960D9680A43DA60EBE7012220388240B7
:103A0000F5E75F28E5D842238022181A413B83401E
:103A1000D205516A99435162516A0B435362D8E708
:103A200010B50400012813D1A022184992050B6893
:103A30005B015B0913430B60154B164A1968114073
:103A4000154A0A431A60402219680A431A6010BDD9
:103A50000028FCD101000A2000F076F821000B209C
:103A600000F072F8C0220A4B920019680A43402104
:103A70001A601A688A431A60B022044912060B6859
:103A80005B015B0913430B60E1E7C04614F00040A3
:103A90001CF000407F00FEFF80FD010072B6074A67
:103AA0001368013313600422054B1A600023054A92
:103AB00013608022D2055360FEE7C0467808FF1FDE
:103AC000C0F00040C4F0004005490B68002B05D150
:103AD000044A0A6004490A60044A13607047C046F9
:103AE000140AFF1F841E0000380AFF1FC4F00040A4
:103AF0000023034A1360034A1360034A13607047AC
:103B000054F0004040F1004044F1004002B47146DE
:103B100049084900095649008E4402BC7047C04616
:103B200002B4714649084900095C49008E4402BC50
:103B30007047C04603B47146490840004900095A1D
:103B400049008E4403BC704701B40248844601BC5E
:103B5000604700BF51A3001101B40248844601BC74
:103B6000604700BF8937010001B40248844601BCA8
:103B7000604700BFF90D010001B40248844601BC52
:103B8000604700BFD1AE000001B40248844601BCCA
:103B9000604700BF6911010001B40248844601BCBE
:103BA000604700BFB352010001B40248844601BC23
:103BB000604700BFCD0C010001B40248844601BC3F
:103BC000604700BF3D71010001B40248844601BC5A
:103BD000604700BF6D0B010001B40248844601BC80
:103BE000604700BFF535010001B40248844601BCBE
:103BF000604700BF6DF6000001B40248844601BC76
:103C0000604700BFE94C010001B40248844601BC92
:103C1000604700BFD5B6001101B40248844601BC1C
:103C2000604700BF7912010001B40248844601BC1C
:103C3000604700BFED68010001B40248844601BC42
:103C4000604700BFC166010001B40248844601BC60
:103C5000604700BF9573010001B40248844601BC6F
:103C6000604700BF4DF9000001B40248844601BC22
:103C7000604700BF19FA000001B40248844601BC45
:103C8000604700BF0534010001B40248844601BC0E
:103C9000604700BFC56D010001B40248844601BC05
:103CA000604700BF090E000001B40248844601BC11
:103CB000604700BF016C010001B40248844601BCAA
:103CC000604700BF090E000001B40248844601BCF1
:103CD000604700BF21A9000001B40248844601BC2E
:103CE000604700BFE90B010001B40248844601BCF3
:103CF000604700BF5976010001B40248844601BC08
:103D0000604700BFC95C010001B40248844601BCA1
:103D1000604700BF0134010001B40248844601BC81
:103D2000604700BF53B9000001B40248844601BC9B
:103D3000604700BF8944000001B40248844601BCCA
:103D4000604700BF496D010001B40248844601BCD0
:103D5000604700BFCD4C010001B40248844601BC5D
:103D6000604700BFE9F6000001B40248844601BC88
:103D7000604700BFB70E000001B40248844601BC92
:103D8000604700BFE9D4000001B40248844601BC8A
:103D9000604700BF85C1000001B40248844601BCF1
:103DA000604700BFEDA5000001B40248844601BC95
:103DB000604700BFDD0C010001B40248844601BC2D
:103DC000604700BFA9D8000001B40248844601BC86
:103DD000604700BFC9A9000001B40248844601BC85
:103DE000604700BF6137010001B40248844601BC4E
:103DF000604700BFC115010001B40248844601BC00
:103E0000604700BFDD0A010001B40248844601BCDE
:103E1000604700BF8512010001B40248844601BC1E
:103E2000604700BF75F8000001B40248844601BC39
:103E3000604700BF2144000001B40248844601BC31
:103E4000604700BFC1A5000001B40248844601BC20
:103E5000604700BFD9B0000001B40248844601BCED
:103E6000604700BFDD3F000001B40248844601BC4A
:103E7000604700BFADAE000001B40248844601BCFB
:103E8000604700BF9DA9000001B40248844601BC00
:103E9000604700BFC1F7000001B40248844601BC7E
:103EA000604700BF0934010001B40248844601BCE8
:103EB000604700BF8914010001B40248844601BC78
:103EC000604700BF8552010001B40248844601BC2E
:103ED000604700BF71B0000001B40248844601BCD5
:103EE000604700BF8B52010001B40248844601BC08
:103EF000604700BF9D6A000001B40248844601BCCF
:103F0000604700BFBD0B010001B40248844601BCFC
:103F1000604700BF2D6C010001B40248844601BC1B
:103F2000604700BFED6B010001B40248844601BC4C
:103F3000604700BF156B010001B40248844601BC14
:103F4000604700BFE512010001B40248844601BC8D
:103F5000604700BFD544010001B40248844601BC5B
:103F6000604700BFE917010001B40248844601BC64
:103F7000604700BFBD5C010001B40248844601BC3B
:103F8000604700BF116E000001B40248844601BCC6
:103F9000604700BF8D11010001B40248844601BC96
:103FA000604700BF0D52010001B40248844601BCC5
:103FB000604700BF01D7000001B40248844601BC3D
:103FC000604700BF8D82000001B40248844601BCF6
:103FD000604700BFE927000001B40248844601BCE5
:103FE000604700BFF9ED000001B40248844601BCFF
:103FF000604700BF75A9000001B40248844601BCB7
:10400000604700BF0167010001B40248844601BC5B
:10401000604700BF0189000001B40248844601BC2A
:10402000604700BF7997000001B40248844601BC94
:10403000604700BFF935010001B40248844601BC65
:08404000604700BF51B8000009
:104048000200000092BF00110100000088BD0011AD
:10405800020000008EBF0011010000008840FF1F11
:104068000200000090BD001101000000C061FF1FA8
:10407800020000008CBF0011030000003461FF1F24
:10408800120000000200000092BF001101000000B1
:10409800D0BD0011020000008EBF00110100000019
:1040A800CDBD001102000000DABD001103000000C0
:1040B8006F61FF1F020000008CBF001103000000A9
:1040C8008461FF1F020000008EBF00110100000084
:1040D800CCBD001102000000D8BD00110300000093
:1040E8004561FF1F020000008CBF001103000000A3
:1040F8006661FF1F0200000092BF0011010000006E
:1041080010BE0011020000008EBF00110100000067
:10411800D141FF1F0200000022BE00110100000073
:104128000BBE0011020000008EBF0011010000004C
:10413800D041FF1F0200000020BE00110100000056
:104148008C61FF1F020000008EBF001101000000FB
:10415800CF41FF1F020000001EBE00110100000039
:10416800FBBD0011020000008EBF0011010000001D
:10417800CE41FF1F020000001CBE0011010000001C
:10418800F6BD0011020000008EBF00110100000002
:10419800CD41FF1F020000001ABE001101000000FF
:1041A800F1BD0011020000008EBF001101000000E7
:1041B800CC41FF1F0200000018BE001101000000E2
:1041C800ECBD001102020202020200000000000021
:1041D8000D0C00009D4C0011634C001180BE0011B5
:1041E80090011D0018001800FFFF070102030405D5
:1041F80006020106000000000000000000000000A8
:1042080000000000000000000000000000000000A6
:10421800030000000200000092BF0011010000002E
:10422800A0BE0011020000008EBF001101000000B6
:104238008C42FF1F02000000AABE0011010000000E
:10424800BA61FF1F020000008CBF001103000000CC
:104258002464FF1F020000008EBF0011010000004F
:104268008C42FF1F02000000A8BE001101000000E0
:10427800BC61FF1F020000008CBF0011030000009A
:104288001C64FF1F126C6C6C00000000005800409A
:10429800151600000001000000000111FFFF0000DA
:1042A8005048593600000000000000000B000500CF
:1042B800F0000000B4000028002800283075A00095
:1042C800A000A000A00000080008E001F000100015
:1042D8001000100010001000100050005000500096
:1042E80010001000D0070000000000000F000100BF
:1042F8000500307507001000010081FF0000000074
:10430800FF0000003975001141730011D1700011D0
:10431800FFFF0100FF000000559F0011D19C001114
:10432800E99B0011000000000000000000000800E8
:10433800040000003B0001085902E0018821280020
:10434800FF0000000200000092BF00110100000001
:1043580058C00011020000008EBF001101000000CB
:10436800C943FF1F020000008ABF001101000000BE
:10437800F067FF1F020000008EBF0011010000005F
:10438800C843FF1F0200000088BF001101000000A1
:10439800C643FF1F020000008EBF0011010000008D
:1043A800C443FF1F0200000086BF00110100000087
:1043B800BC43FF1F180018001D00900102000003F5
:1043C800020200000200000092BF0011010000007C
:1043D8006CC00011020000008EBF00110100000037
:1043E8000C44FF1F0200000084BF00110000000001
:1043F80000000000020000008CBF00110300000054
:064408001068FF1F20FFF9
:040000051FFF184180
:00000001FF
